:020000040000FA
:040800003CEF0CF0CD
:1008100003B275EF05F0F2B493EF05F09EB09BEFD5
:1008200005F09EB2A3EF05F0F2A81AEF04F0F2B2C1
:1008300023EF04F0F2B01FEF04F0EBEF0BF0F296B1
:10084000F290EBEF0BF0CD90F2929EA02DEF04F022
:100850000101533F2DEF04F0542BB2C1B6F1B3C1E7
:10086000B7F1B4C1B8F1B5C1B9F1AEC1B2F1AFC120
:10087000B3F1B0C1B4F1B1C1B5F1AAC1AEF1ABC130
:10088000AFF1ACC1B0F1ADC1B1F1A6C1AAF1A7C140
:10089000ABF1A8C1ACF1A9C1ADF1A2C1A6F1A3C150
:1008A000A7F1A4C1A8F1A5C1A9F19EC1A2F19FC160
:1008B000A3F1A0C1A4F1A1C1A5F19AC19EF19BC170
:1008C0009FF19CC1A0F19DC1A1F1CECF9AF1CFCFF4
:1008D0009BF153C19CF154C19DF1CF6ACE6A0101D5
:1008E000536B546B9E90CD800FBC0F8E0FBA7CEF74
:1008F00004F00F8AEBEF0BF013880F8C0FBEB9EFEB
:1009000004F09AC19EF19BC19FF19CC1A0F19DC1D1
:10091000A1F19EC1A2F19FC1A3F1A0C1A4F1A1C107
:10092000A5F1A2C1A6F1A3C1A7F1A4C1A8F1A5C1D7
:10093000A9F1A6C1AAF1A7C1ABF1A8C1ACF1A9C1A7
:10094000ADF1AAC1AEF1ABC1AFF1ACC1B0F1ADC177
:10095000B1F1AEC1B2F1AFC1B3F1B0C1B4F1B1C147
:10096000B5F1B2C1B6F1B3C1B7F1B4C1B8F1B5C117
:10097000B9F101015E6B5F6B606B616B9A515E2731
:100980009B515F239C5160239D5161239E515E27A3
:100990009F515F23A0516023A1516123A2515E2783
:1009A000A3515F23A4516023A5516123A6515E2763
:1009B000A7515F23A8516023A9516123AA515E2743
:1009C000AB515F23AC516023AD516123AE515E2723
:1009D000AF515F23B0516023B1516123B2515E2703
:1009E000B3515F23B4516023B5516123B6515E27E3
:1009F000B7515F23B8516023B9516123D8900101E9
:100A0000613360335F335E33D8900101613360330B
:100A10005F335E33D8900101613360335F335E33FF
:100A200000C10CF101C10DF102C10EF103C10FF1C2
:100A300004C110F105C111F106C112F107C113F192
:100A400008C114F109C115F10AC116F10BC117F162
:100A500034C135F111B838EF05F00101620E046FB1
:100A6000010E056F000E066F000E076F41EF05F0D7
:100A70000101A70E046F020E056F000E066F000E37
:100A8000076F5EC100F15FC101F160C102F161C198
:100A900003F1F2EC3AF003BF04D01CBE02D01CA05C
:100AA000108C11A059EF05F010BA59EF05F00F8026
:100AB000108A0CC100F10DC101F10EC102F10FC18C
:100AC00003F110C104F111C105F112C106F113C106
:100AD00007F114C108F115C109F116C10AF117C1D6
:100AE0000BF135C134F1EBEF0BF00392ABB2AB98E5
:100AF000AB88030103EE00F080517F0BE92604C0B0
:100B0000EFFF802B8151805D700BD8A48B82000099
:100B10008051815D700BD8A48B9281518019D8B41B
:100B20000790EBEF0BF0F2940101453FEBEF0BF078
:100B3000462BEBEF0BF09E900101533FEBEF0BF0D8
:100B4000542BEBEF0BF09E9211B895EF08F00400D8
:100B500066A1ABEF05F08BB4B5EF05F010ACB5EFC7
:100B600005F08B84109CB6EF05F08B9407B408EF6A
:100B700006F007B008EF06F01EC620F61FC621F6E5
:100B80001CC61EF61DC61FF61AC61CF61BC61DF691
:100B900006C608F607C609F604C606F605C607F631
:100BA00002C604F603C605F626C628F627C629F6A9
:100BB00024C626F625C627F622C624F623C625F621
:100BC0000EC610F60FC611F60CC60EF60DC60FF6C1
:100BD0000AC60CF60BC60DF62EC630F62FC631F639
:100BE0002CC62EF62DC62FF62AC62CF62BC62DF6B1
:100BF00016C618F617C619F614C616F615C617F651
:100C000012C614F613C615F606EC3DF0B4EC3CF033
:100C1000077C07AC23EF06F0C274C2B41DEF06F0E8
:100C2000C3CFB7F5C4CFB8F50501D890B833B73303
:100C3000D890B833B73324EF06F0C3CF55F1C4CF03
:100C400056F124EF06F0C28207B496EF06F047C1D2
:100C50004BF148C14CF149C14DF14AC14EF15EC161
:100C600062F15FC163F160C164F161C165F113A814
:100C70003CEF06F0138C13989AC1BAF19BC1BBF1FB
:100C80009CC1BCF19DC1BDF19EC1BEF19FC1BFF130
:100C9000A0C1C0F1A1C1C1F1A2C1C2F1A3C1C3F100
:100CA000A4C1C4F1A5C1C5F1A6C1C6F1A7C1C7F1D0
:100CB000A8C1C8F1A9C1C9F1AAC1CAF1ABC1CBF1A0
:100CC000ACC1CCF1ADC1CDF1AEC1CEF1AFC1CFF170
:100CD000B0C1D0F1B1C1D1F1B2C1D2F1B3C1D3F140
:100CE000B4C1D4F1B5C1D5F1B6C1D6F1B7C1D7F110
:100CF000B8C1D8F1B9C1D9F1B7C5B9F5B8C5BAF518
:100D0000B9C5BBF5BAC5BCF5010155515B275651B4
:100D10005C23E86A5D230E2E96EF06F05CC157F166
:100D20005DC158F15B6B5C6B5D6B078E0201002F40
:100D3000EBEF0BF03C0E006F1D50E00BE00AE86695
:100D400012881BBE02D01BB4108E00C10CF101C171
:100D50000DF102C10EF103C10FF104C110F105C183
:100D600011F106C112F107C113F108C114F109C153
:100D700015F10AC116F10BC117F134C135F181AA81
:100D8000FEEF06F015A449EF07F005012F51000A08
:100D9000D8B48CEF07F005012F51010AD8B408EF41
:100DA00007F005012F51020AD8B449EF07F00501F9
:100DB0002F51030AD8B449EF07F005012F51040A57
:100DC000D8B449EF07F005012F51050AD8B449EF0F
:100DD00007F005012F51060AD8B449EF07F00501C5
:100DE0002F51070AD8B449EF07F005012F51320AF5
:100DF000D8B406EF07F02F6B8CEF07F00001165008
:100E0000030AD8B449EF07F08CEF07F08CEF07F036
:100E10000501576713EF07F0586713EF07F059679D
:100E200013EF07F05A6717EF07F08CEF07F05BC579
:100E300000F15CC501F15DC502F15EC503F1010180
:100E4000010E046F000E056F000E066F000E076F97
:100E5000F2EC3AF000C15BF501C15CF502C15DF551
:100E600003C15EF5010100673DEF07F001673DEF4B
:100E700007F002673DEF07F003678CEF07F057C5F7
:100E80005BF558C55CF559C55DF55AC55EF576EF5D
:100E900007F00FBE5EEF07F010A063EF07F001014F
:100EA00047675AEF07F048675AEF07F049675AEF6C
:100EB00007F04A675EEF07F063EF07F007AE63EFF6
:100EC00007F076EF07F00501312F8CEF07F03C0EAD
:100ED000316F302F8CEF07F00101000E626FE00ED2
:100EE000636FA50E646F010E656F138800011650C5
:100EF000000AD8B484EF07F000011650030AD8B4F2
:100F000089EF07F08CEF07F00001010E166E8CEFF1
:100F100007F00001040E166E0501666B37B792EFFD
:100F200007F066810CC100F10DC101F10EC102F1A3
:100F30000FC103F110C104F111C105F112C106F195
:100F400013C107F114C108F115C109F116C10AF165
:100F500017C10BF135C134F100C10CF101C10DF124
:100F600002C10EF103C10FF104C110F105C111F16D
:100F700006C112F107C113F108C114F109C115F13D
:100F80000AC116F10BC117F134C135F101018E67A9
:100F9000D1EF07F08F67D1EF07F09067D1EF07F03F
:100FA0009167D5EF07F006EF08F092C100F193C109
:100FB00001F194C102F195C103F10101010E046F29
:100FC000000E056F000E066F000E076FF2EC3AF090
:100FD00000C192F101C193F102C194F103C195F1F5
:100FE00001010067FBEF07F00167FBEF07F0026705
:100FF000FBEF07F0036706EF08F08EC192F18FC197
:1010000093F190C194F191C195F10F80D57ED5BE39
:101010006ED0D6CF47F1D7CF48F145C149F1E86A44
:10102000E8CF4AF1138A1CBE02D01CA0108C10908D
:1010300047C100F148C101F149C102F14AC103F1C0
:1010400001010A0E046F000E056F000E066F000E00
:10105000076FF2EC3AF003AF1080010154A73DEFA7
:1010600008F00F9A0F9C0F9E0101000E5E6F600E3C
:101070005F6F3D0E606F080E616F010147BF4DEF5E
:1010800008F048674DEF08F049674DEF08F04A67F0
:101090004DEF08F0F28872EF08F0F2985E6B5F6B2C
:1010A000606B616B9A6B9B6B9C6B9D6B9E6B9F6B7C
:1010B000A06BA16BA26BA36BA46BA56BA66BA76BBC
:1010C000A86BA96BAA6BAB6BAC6BAD6BAE6BAF6B6C
:1010D000B06BB16BB26BB36BB46BB56BB66BB76B1C
:1010E000B86BB96BD76AD66A0101456B466B0CC108
:1010F00000F10DC101F10EC102F10FC103F110C1E8
:1011000004F111C105F112C106F113C107F114C1B7
:1011100008F115C109F116C10AF117C10BF135C16A
:1011200034F1EBEF0BF0EBEF0BF00201002FFDEFD2
:101130000AF0D59ED6CF47F1D7CF48F145C149F146
:10114000E86AE8CF4AF1138AD76AD66A0101456B8B
:10115000466BD58E1D50E00BE00AE86612881BBE78
:1011600002D01BB4108E1AAE1F8C00C10CF101C14D
:101170000DF102C10EF103C10FF104C110F105C15F
:1011800011F106C112F107C113F108C114F109C12F
:1011900015F10AC116F10BC117F134C135F10FA0D9
:1011A000109A11B8DFEF08F00101620E046F010E12
:1011B000056F000E066F000E076FE8EF08F00101E3
:1011C000A70E046F020E056F000E066F000E076F6C
:1011D00047C100F148C101F149C102F14AC103F11F
:1011E000F2EC3AF003BFFBEF08F01CBE02D01CA0EB
:1011F000108C11B00F800CC100F10DC101F10EC1B6
:1012000002F10FC103F110C104F111C105F112C1C6
:1012100006F113C107F114C108F115C109F116C196
:101220000AF117C10BF135C134F102013C0E006F18
:1012300000C10CF101C10DF102C10EF103C10FF1AA
:1012400004C110F105C111F106C112F107C113F17A
:1012500008C114F109C115F10AC116F10BC117F14A
:1012600034C135F181BA38EF09F015B277EF09F0E2
:1012700015A077EF09F015A4C2EF09F005012F5171
:10128000000AD8B405EF0AF005012F51010AD8B4BD
:1012900081EF09F005012F51020AD8B4C2EF09F01D
:1012A00005012F51030AD8B4C2EF09F005012F51EF
:1012B000040AD8B4C2EF09F005012F51050AD8B4C9
:1012C000C2EF09F005012F51060AD8B4C2EF09F0A8
:1012D00005012F51070AD8B4C2EF09F005012F51BB
:1012E000320AD8B47FEF09F02F6B05EF0AF0000146
:1012F0001650030AD8B4C2EF09F005EF0AF005EF63
:101300000AF0050157678CEF09F058678CEF09F078
:1013100059678CEF09F05A6790EF09F005EF0AF072
:101320005BC500F15CC501F15DC502F15EC503F16D
:101330000101010E046F000E056F000E066F000E16
:10134000076FF2EC3AF000C15BF501C15CF502C138
:101350005DF503C15EF501010067B6EF09F00167B5
:10136000B6EF09F00267B6EF09F0036705EF0AF080
:1013700057C55BF558C55CF559C55DF55AC55EF5B1
:10138000EFEF09F00FBED7EF09F010A0DCEF09F086
:1013900001014767D3EF09F04867D3EF09F04967C8
:1013A000D3EF09F04A67D7EF09F0DCEF09F007AE99
:1013B000DCEF09F0EFEF09F00501312F05EF0AF03E
:1013C0003C0E316F302F05EF0AF00101000E626F05
:1013D000E00E636FA50E646F010E656F1388000148
:1013E0001650000AD8B4FDEF09F000011650030AA8
:1013F000D8B402EF0AF005EF0AF00001010E166EF4
:1014000005EF0AF00001040E166E0501666B37B792
:101410000BEF0AF066810CC100F10DC101F10EC1A4
:1014200002F10FC103F110C104F111C105F112C1A4
:1014300006F113C107F114C108F115C109F116C174
:101440000AF117C10BF135C134F100C10CF101C132
:101450000DF102C10EF103C10FF104C110F105C17C
:1014600011F106C112F107C113F108C114F109C14C
:1014700015F10AC116F10BC117F134C135F10101A3
:101480008E674AEF0AF08F674AEF0AF090674AEFDB
:101490000AF091674EEF0AF07FEF0AF092C100F177
:1014A00093C101F194C102F195C103F10101010E53
:1014B000046F000E056F000E066F000E076FF2EC52
:1014C0003AF000C192F101C193F102C194F103C15C
:1014D00095F10101006774EF0AF0016774EF0AF0FB
:1014E000026774EF0AF003677FEF0AF08EC192F192
:1014F0008FC193F190C194F191C195F10F8010903B
:1015000047C100F148C101F149C102F14AC103F1EB
:1015100001010A0E046F000E056F000E066F000E2B
:10152000076FF2EC3AF003AF1080010154A7A5EF6A
:101530000AF00F9A0F9C0F9E0101000E5E6F600E65
:101540005F6F3D0E606F080E616F47C100F148C1CB
:1015500001F149C102F14AC103F10101140E046F06
:10156000050E056F000E066F000E076FF2EC3AF0E5
:1015700003AFBEEF0AF0F288E3EF0AF0F2985E6B79
:101580005F6B606B616B9A6B9B6B9C6B9D6B9E6BD7
:101590009F6BA06BA16BA26BA36BA46BA56BA66BDF
:1015A000A76BA86BA96BAA6BAB6BAC6BAD6BAE6B8F
:1015B000AF6BB06BB16BB26BB36BB46BB56BB66B3F
:1015C000B76BB86BB96B0CC100F10DC101F10EC165
:1015D00002F10FC103F110C104F111C105F112C1F3
:1015E00006F113C107F114C108F115C109F116C1C3
:1015F0000AF117C10BF135C134F104008BB408EFC7
:101600000BF010AC08EF0BF08B84109C09EF0BF083
:101610008B9407B45BEF0BF007B05BEF0BF01EC6CB
:1016200020F61FC621F61CC61EF61DC61FF61AC6DA
:101630001CF61BC61DF606C608F607C609F604C644
:1016400006F605C607F602C604F603C605F626C664
:1016500028F627C629F624C626F625C627F622C66A
:1016600024F623C625F60EC610F60FC611F60CC6D4
:101670000EF60DC60FF60AC60CF60BC60DF62EC6F4
:1016800030F62FC631F62CC62EF62DC62FF62AC6FA
:101690002CF62BC62DF616C618F617C619F614C664
:1016A00016F615C617F612C614F613C615F606EC8E
:1016B0003DF0B4EC3CF0077C07AC76EF0BF0C27465
:1016C000C2B470EF0BF0C3CFB7F5C4CFB8F50501C6
:1016D000D890B833B733D890B833B73377EF0BF02F
:1016E000C3CF55F1C4CF56F177EF0BF0C28207B4E8
:1016F000E9EF0BF047C14BF148C14CF149C14DF145
:101700004AC14EF15EC162F15FC163F160C164F133
:1017100061C165F113A88FEF0BF0138C13989AC178
:10172000BAF19BC1BBF19CC1BCF19DC1BDF19EC191
:10173000BEF19FC1BFF1A0C1C0F1A1C1C1F1A2C161
:10174000C2F1A3C1C3F1A4C1C4F1A5C1C5F1A6C131
:10175000C6F1A7C1C7F1A8C1C8F1A9C1C9F1AAC101
:10176000CAF1ABC1CBF1ACC1CCF1ADC1CDF1AEC1D1
:10177000CEF1AFC1CFF1B0C1D0F1B1C1D1F1B2C1A1
:10178000D2F1B3C1D3F1B4C1D4F1B5C1D5F1B6C171
:10179000D6F1B7C1D7F1B8C1D8F1B9C1D9F1B7C540
:1017A000B9F5B8C5BAF5B9C5BBF5BAC5BCF50101FF
:1017B00055515B2756515C23E86A5D230E2EE9EFF5
:1017C0000BF05CC157F15DC158F15B6B5C6B5D6BFD
:1017D000078EEBEF0BF002C0E0FF005001C0D8FF16
:1017E0001000A6B2F1EF0BF00CC0A9FF0BC0A8FFD0
:1017F000A69EA69CA684F29E550EA76EAA0EA76E64
:10180000A682F28EA694A6B203EF0CF00C2A120068
:10181000A96EA69EA69CA680A8500C2A12000401C0
:101820002C0E826F70EC0FF007EC3CF00C5008ECC3
:101830000CF0E8CF00F10C5008EC0CF0E8CF01F10F
:1018400001AF28EF0CF00101FF0E026FFF0E036FD6
:1018500090EC3BF0296734EF0CF00401200E826F0E
:1018600070EC0FF039EF0CF004012D0E826F70EC6C
:101870000FF09AEC39F0120015941596076A0F6A6A
:10188000106A116A126A136A166A0F010D0EC16E90
:10189000860EC06E030EC26E0F01680E896E130EA7
:1018A000926E080E8A6E8A6AF30E936E8B6A900EA1
:1018B000946EC80E08EC0CF0E8CFE8FF1098E8A092
:1018C000108810A805D00E0E256E8E0E266E04D040
:1018D0000F0E256E8F0E266ED7EC3DF022EC3FF0FA
:1018E000F18EF19EFC0E08EC0CF0E8CF0BF00BA093
:1018F00011800BA211820BA411840BA81188C90EB0
:1019000008EC0CF0E8CF1AF0CA0E08EC0CF0E8CFA7
:101910001BF0CB0E08EC0CF0E8CF1CF0CC0E08EC62
:101920000CF0E8CF1DF0FB0E08EC0CF0E8CF37F020
:10193000CE0E08EC0CF0E8CF14F0CD0E08EC0CF055
:10194000E8CF36F01F6A206A0E6A01015B6B5C6BA0
:101950005D6B576B586BF29A0101476B486B496B93
:101960004A6B4B6B4C6B4D6B4E6B4F6B506B516BB3
:10197000526B456B466BD76AD66A0F01280ED56E3F
:10198000F28A9D90B00ECD6E01015E6B5F6B606B55
:10199000616B626B636B646B656B666B676B686BCB
:1019A000696B536B546BCF6ACE6A0F9A0F9C0F9E74
:1019B0009D80760ECA6E9D8202013C0E006FCC6A3D
:1019C000160E08EC0CF0E8CF00F1170E08EC0CF046
:1019D000E8CF01F1180E08EC0CF0E8CF02F1190E77
:1019E00008EC0CF0E8CF03F1010103AF12EF0DF0AA
:1019F00007EC3CF0160E0C6E00C10BF0F1EC0BF096
:101A0000170E0C6E01C10BF0F1EC0BF0180E0C6E02
:101A100002C10BF0F1EC0BF0190E0C6E03C10BF0D0
:101A2000F1EC0BF000C18EF101C18FF102C190F118
:101A300003C191F100C192F101C193F102C194F18E
:101A400003C195F11A0E08EC0CF0E8CF00F11B0E63
:101A500008EC0CF0E8CF01F11C0E08EC0CF0E8CF1C
:101A600002F11D0E08EC0CF0E8CF03F1010103AF09
:101A700068EF0DF007EC3CF01A0E0C6E00C10BF095
:101A8000F1EC0BF01B0E0C6E01C10BF0F1EC0BF046
:101A90001C0E0C6E02C10BF0F1EC0BF01D0E0C6E67
:101AA00003C10BF0F1EC0BF01A0E08EC0CF0E8CFD0
:101AB00000F11B0E08EC0CF0E8CF01F11C0E08EC55
:101AC0000CF0E8CF02F11D0E08EC0CF0E8CF03F1AA
:101AD00000C196F101C197F102C198F103C199F1DA
:101AE000240EAC6E900EAB6E240EAC6E080EB86E6B
:101AF000000EB06E1F0EAF6E0401806B816B0F0184
:101B0000900EAB6E0F019D8A0301806B816BC26BDF
:101B10008B927CEC42F07CEC42F0880E08EC0CF0EE
:101B2000E8CF00F1890E08EC0CF0E8CF01F10101DB
:101B300001AFB3EF0DF007EC3CF0880E0C6E00C166
:101B40000BF0F1EC0BF0890E0C6E01C10BF0F1EC17
:101B50000BF0880E08EC0CF0E8CF00F1890E08ECD1
:101B60000CF0E8CF01F100C140F601C141F602C11D
:101B700042F603C143F65AEC46F05AEC40F0200E10
:101B800008EC0CF0E8CF2FF505012F51FF0AD8A47F
:101B9000D1EF0DF02F6B200E0C6E2FC50BF0F1EC7A
:101BA0000BF00501010E306F3C0E316F250E08EC75
:101BB0000CF0E8CF00F1260E08EC0CF0E8CF01F1B4
:101BC000270E08EC0CF0E8CF02F1280E08EC0CF020
:101BD000E8CF03F1010103AF08EF0EF007EC3CF092
:101BE000250E0C6E00C10BF0F1EC0BF0260E0C6E06
:101BF00001C10BF0F1EC0BF0270E0C6E02C10BF0E3
:101C0000F1EC0BF0280E0C6E03C10BF0F1EC0BF0B5
:101C100000C157F501C158F502C159F503C15AF584
:101C200000C15BF501C15CF502C15DF503C15EF564
:101C3000290E08EC0CF0E8CF5FF5050160515F5DFF
:101C4000D8A05FC560F5210E08EC0CF0E8CF00F1DC
:101C5000220E08EC0CF0E8CF01F1230E08EC0CF09A
:101C6000E8CF02F1240E08EC0CF0E8CF03F10101FB
:101C700003AF69EF0EF007EC3CF0210E0C6E00C1D3
:101C80000BF0F1EC0BF0220E0C6E01C10BF0F1EC3D
:101C90000BF0230E0C6E02C10BF0F1EC0BF0240ED6
:101CA0000C6E03C10BF0F1EC0BF0210E08EC0CF004
:101CB000E8CF00F1220E08EC0CF0E8CF01F1230E82
:101CC00008EC0CF0E8CF02F1240E08EC0CF0E8CFA1
:101CD00003F100C161F501C162F502C163F503C101
:101CE00064F5A2EC3FF088EC3EF0E0EC3DF015909E
:101CF000C70E08EC0CF0E8CF00F1010100B184EF51
:101D00000EF0159285EF0EF0158281AA93EF0EF07A
:101D100015B48EEF0EF0158093EF0EF099EC46F0AF
:101D200015A000EF47F058EC3DF007900001F28E4F
:101D3000F28C12AE03D012BC1CEF21F007B02CEFD6
:101D400037F00FB01CEF30F010BE1CEF30F012B8BF
:101D50001CEF30F000011650010AD8B424EF27F030
:101D600081BABBEF0EF000011650040AD8B4C8EFD8
:101D700023F0C1EF0EF000011650040AD8B460EF52
:101D800027F00301805181197F0BD8B42CEF37F075
:101D900013EE00F081517F0BE126812BE7CFE8FFA6
:101DA000E00BD8B42CEF37F023EE82F0C2513F0B9A
:101DB000D926E7CFDFFFC22BDF50780AD8A42CEF5B
:101DC00037F0078092C100F193C101F194C102F193
:101DD00095C103F10101040E046F000E056F000EA2
:101DE000066F000E076FF2EC3AF000AF01EF0FF054
:101DF0000101030E926F000E936F000E946F000EA0
:101E0000956F03018251720AD8B49DEF2FF0825171
:101E1000520AD8B49DEF2FF08251750AD8B49DEFC5
:101E20002FF08251680AD8B484EF0FF08251630A10
:101E3000D8B4E6EF33F08251690AD8B46AEF2AF0D9
:101E400082517A0AD8B47DEF2BF08251490AD8B476
:101E500009EF2AF08251500AD8B427EF29F08251B5
:101E6000700AD8B46AEF29F08251540AD8B495EFB9
:101E700029F08251740AD8B4DBEF29F08251410A6B
:101E8000D8B489EF10F082514B0AD8B486EF0FF026
:101E900082516D0AD8B4F9EF14F082514D0AD8B4CA
:101EA00012EF15F08251730AD8B4CDEF2EF08251A3
:101EB000530AD8B432EF2FF082514C0AD8B475EFE0
:101EC0001CF08251760AD8B4A1EF15F08251590A5C
:101ED000D8B44AEF14F012AE01D0128C1DEF34F0DA
:101EE000040114EE00F080517F0BE12682C4E7FF6D
:101EF000802B120004010D0E826F70EC0FF00A0EA1
:101F0000826F70EC0FF012001BEF34F004014B0EE7
:101F1000826F70EC0FF004012C0E826F70EC0FF0EA
:101F200081B802D036B630D003018351430AD8B409
:101F3000CBEF0FF003018351630AD8B4CDEF0FF05C
:101F400003018351520AD8B4CFEF0FF0030183513C
:101F5000720AD8B4D1EF0FF003018351470AD8B405
:101F6000D3EF0FF003018351670AD8B4D5EF0FF018
:101F700003018351540AD8B4D7EF0FF00301835102
:101F8000740AD8B447EF10F003018351550AD8B44E
:101F9000D9EF0FF083D036807BD0369079D036825F
:101FA00077D0369275D0368473D0369471D0368619
:101FB0006FD084C330F185C331F186C332F187C35A
:101FC00033F10101296B55EC3CF0CCEC3BF000C146
:101FD00004F101C105F102C106F103C107F148ECAA
:101FE0003CF0200EF86EF76AF66A0900F5CF2CF186
:101FF0000900F5CF2DF10900F5CF2EF10900F5CF3D
:102000002FF10900F5CF30F10900F5CF31F10900CA
:10201000F5CF32F10900F5CF33F10101296B55EC11
:102020003CF0CCEC3BF0F2EC3AF00101006720EF21
:1020300010F0016720EF10F0026720EF10F0036747
:1020400001D025D004014E0E826F70EC0FF0040118
:102050006F0E826F70EC0FF004014D0E826F70EC0A
:102060000FF00401610E826F70EC0FF00401740E2A
:10207000826F70EC0FF00401630E826F70EC0FF052
:102080000401680E826F70EC0FF01BEF34F036968F
:10209000CD0E0C6E36C00BF0F1EC0BF0CD0E08EC53
:1020A0000CF0E8CF36F036B006D00401630E826F34
:1020B00070EC0FF005D00401430E826F70EC0FF04E
:1020C00036B206D00401720E826F70EC0FF005D0AC
:1020D0000401520E826F70EC0FF036B406D004018A
:1020E000670E826F70EC0FF005D00401470E826F0F
:1020F00070EC0FF036B606D00401740E826F70ECEF
:102100000FF005D00401540E826F70EC0FF01BEF3E
:1021100034F00401410E826F70EC0FF00301835123
:10212000310AD8B46AEF13F003018351320AD8B4EC
:102130009AEF12F003018351330AD8B423EF12F05F
:1021400003018351340AD8B413EF11F00301835112
:10215000350AD8B4B3EF10F004013F0E826F70EC73
:102160000FF01BEF34F003018451300AD8B4D9EFDB
:1021700010F003018451310AD8B4DCEF10F00301F0
:102180008451650AD8B4CDEF10F003018451640A7C
:10219000D8B4D0EF10F0DDEF10F03790D1EF10F0A1
:1021A0003780FB0E0C6E37C00BF0F1EC0BF0DDEF5F
:1021B00010F08B90DDEF10F08B800401350E826FF4
:1021C00070EC0FF004012C0E826F70EC0FF08BB0EE
:1021D000F1EF10F00401300E826F70EC0FF0F6EFAB
:1021E00010F00401310E826F70EC0FF004012C0E20
:1021F000826F70EC0FF0FB0E08EC0CF0E8CF37F0BC
:1022000037A00AEF11F00401640E826F70EC0FF03A
:102210000FEF11F00401650E826F70EC0FF011EFFB
:1022200011F01BEF34F0CC0E08EC0CF0E8CF0BF003
:1022300004012C0E826F70EC0FF003018451310AFF
:10224000D8B437EF11F003018451300AD8B439EF14
:1022500011F0030184514D0AD8B443EF11F003018A
:102260008451540AD8B44AEF11F061EF11F08A8416
:1022700001D08A940BAE04D00BAC02D00BBA21D0A3
:10228000E00E0B1218D01F0E0B168539E844E00B38
:102290000B1211D0E00E0B1648EC3CF085C332F166
:1022A00086C333F10101296B55EC3CF0CCEC3BF0DB
:1022B00000511F0B0B12CC0E0C6E0BC00BF0F1EC8F
:1022C0000BF00401340E826F70EC0FF004012C0E41
:1022D000826F70EC0FF0CC0E08EC0CF0E8CF1DF024
:1022E0008AB406D00401300E826F70EC0FF005D076
:1022F0000401310E826F70EC0FF004012C0E826F1E
:1023000070EC0FF01D38E840070BE8CF82F40401B1
:10231000300E822770EC0FF004012C0E826F70ECEF
:102320000FF007EC3CF01D501F0BE8CF00F190ECD4
:102330003BF032C182F40401300E822770EC0FF0C2
:1023400033C182F40401300E822770EC0FF00401D7
:102350002C0E826F70EC0FF007EC3CF030C000F1F7
:1023600000AF0BD0FF0E016FFF0E026FFF0E036F69
:1023700004012D0E826F70EC0FF090EC3BF031C138
:1023800082F40401300E822770EC0FF032C182F427
:102390000401300E822770EC0FF033C182F4040187
:1023A000300E822770EC0FF004012C0E826F70EC5F
:1023B0000FF007EC3CF02FC000F190EC3BF031C186
:1023C00082F40401300E822770EC0FF032C182F4E7
:1023D0000401300E822770EC0FF033C182F4040147
:1023E000300E822770EC0FF004012C0E826F70EC1F
:1023F0000FF007EC3CF031C000F100AF0BD0FF0E46
:10240000016FFF0E026FFF0E036F04012D0E826F2E
:1024100070EC0FF090EC3BF031C182F40401300E0F
:10242000822770EC0FF032C182F40401300E822753
:1024300070EC0FF033C182F40401300E822770EC8F
:102440000FF01BEF34F0CB0E08EC0CF0E8CF0BF0E4
:1024500004012C0E826F70EC0FF003018451450AC9
:10246000D8B447EF12F003018451440AD8B44AEFBC
:1024700012F003018451300AD8B44DEF12F0030179
:102480008451310AD8B451EF12F05CEF12F00B9E78
:1024900056EF12F00B8E56EF12F0FC0E0B1656EFA5
:1024A00012F0FC0E0B160B8056EF12F0CB0E0C6EDA
:1024B0000BC00BF0F1EC0BF00401330E826F70ECEB
:1024C0000FF004012C0E826F70EC0FF0CB0E08ECB5
:1024D0000CF0E8CF1CF01CBE75EF12F00401450EA5
:1024E000826F70EC0FF07AEF12F00401440E826FED
:1024F00070EC0FF004012C0E826F70EC0FF00401F1
:10250000300E826F70EC0FF004012C0E826F70ECB5
:102510000FF01CB093EF12F00401300E826F70ECDC
:102520000FF098EF12F00401310E826F70EC0FF093
:102530001BEF34F0CA0E08EC0CF0E8CF0BF00401EE
:102540002C0E826F70EC0FF003018451450AD8B451
:10255000D6EF12F003018451440AD8B4D9EF12F037
:10256000030184514D0AD8B4E2EF12F00301845103
:10257000410AD8B4DCEF12F003018451460AD8B402
:10258000DFEF12F003018451560AD8B4EAEF12F0DB
:1025900003018451500AD8B4F5EF12F003018451BD
:1025A000520AD8B4F8EF12F001EF13F00B9EFBEFD4
:1025B00012F00B8EFBEF12F00B9CFBEF12F00B8C6A
:1025C000FBEF12F0FC0E0B1685C3E8FF030B0B129A
:1025D000FBEF12F0C70E0B1685C3E8FF070BE846AA
:1025E000E846E8460B12FBEF12F00B84FBEF12F00B
:1025F0000B94FBEF12F0CA0E0C6E0BC00BF0F1EC5B
:102600000BF0CA0E08EC0CF0E8CF1BF00401320E00
:10261000826F70EC0FF004012C0E826F70EC0FF0E3
:102620001BBE1AEF13F00401450E826F70EC0FF021
:102630001FEF13F00401440E826F70EC0FF00401E1
:102640002C0E826F70EC0FF01BC0E8FF030BE8CF7D
:1026500082F40401300E822770EC0FF004012C0E7E
:10266000826F70EC0FF01BBC3DEF13F00401410EC4
:10267000826F70EC0FF042EF13F00401460E826F90
:1026800070EC0FF004012C0E826F70EC0FF01BC089
:10269000E8FF380BE842E842E842E8CF82F4040160
:1026A000300E822770EC0FF004012C0E826F70EC5C
:1026B0000FF01BB463EF13F00401520E826F70EC45
:1026C0000FF068EF13F00401500E826F70EC0FF002
:1026D0001BEF34F0C90E08EC0CF0E8CF0BF004014E
:1026E0002C0E826F70EC0FF003018451450AD8B4B0
:1026F00088EF13F003018451440AD8B48BEF13F030
:10270000030184514D0AD8B48EEF13F09CEF13F0FF
:102710000B9E96EF13F00B8E96EF13F0F80E0B1640
:1027200085C3E8FF070B0B1296EF13F0C90E0C6E72
:102730000BC00BF0F1EC0BF00401310E826F70EC6A
:102740000FF004012C0E826F70EC0FF0C90E08EC34
:102750000CF0E8CF1AF01ABE06D00401450E826FC5
:1027600070EC0FF005D00401440E826F70EC0FF096
:1027700004012C0E826F70EC0FF01AC0E8FF070BFB
:10278000E8CF82F40401300E822770EC0FF00401D0
:102790002C0E826F70EC0FF0078007EC3CF02BC022
:1027A000E8FF003B00430043030B90EC3BF033C1D8
:1027B00082F40401300E822770EC0FF004012C0E1D
:1027C000826F70EC0FF007EC3CF02BC001F1019F21
:1027D000019D2CC000F1010190EC3BF02FC182F46F
:1027E0000401300E822770EC0FF030C182F4040136
:1027F000300E822770EC0FF031C182F40401300EEC
:10280000822770EC0FF032C182F40401300E82276F
:1028100070EC0FF033C182F40401300E822770ECAB
:102820000FF004012C0E826F70EC0FF007EC3CF0FF
:102830002DC001F12EC000F1D89001330033D890A3
:1028400001330033010190EC3BF02FC182F404010D
:10285000300E822770EC0FF030C182F40401300E8C
:10286000822770EC0FF031C182F40401300E822710
:1028700070EC0FF032C182F40401300E822770EC4C
:102880000FF033C182F40401300E822770EC0FF098
:102890001BEF34F0FC0E08EC0CF0E8CF0BF003015A
:1028A0008351520AD8B481EF14F003018351720AA4
:1028B000D8B484EF14F003018351500AD8B487EFE1
:1028C00014F003018351700AD8B48AEF14F00301A5
:1028D0008351550AD8B48DEF14F003018351750A62
:1028E000D8B490EF14F003018351430AD8B499EFA0
:1028F00014F003018351630AD8B49CEF14F0A5EFE0
:1029000014F00B909FEF14F00B809FEF14F00B92DC
:102910009FEF14F00B829FEF14F00B949FEF14F0D5
:102920000B849FEF14F00B969FEF14F00B869FEF34
:1029300014F00B989FEF14F00B889FEF14F0FC0E2F
:102940000C6E0BC00BF0F1EC0BF00401590E826F12
:1029500070EC0FF01190119211941198FC0E08EC8C
:102960000CF0E8CF0BF00BA011800BA211820BA48E
:1029700011840BA8118811A0C5EF14F00401520EA8
:10298000826F70EC0FF0CAEF14F00401720E826FC8
:1029900070EC0FF011A8D4EF14F00401430E826F15
:1029A00070EC0FF0D9EF14F00401630E826F70EC3D
:1029B0000FF011A2E3EF14F00401500E826F70ECDF
:1029C0000FF0E8EF14F00401700E826F70EC0FF05E
:1029D00011A4F2EF14F00401550E826F70EC0FF0A9
:1029E000F7EF14F00401750E826F70EC0FF01BEF1F
:1029F00034F004016D0E826F70EC0FF0030183510F
:102A0000300AD8B451EF15F003018351310AD8B41C
:102A100064EF15F003018351320AD8B477EF15F053
:102A20001DEF34F004014D0E826F70EC0FF048EC96
:102A30003CF084C331F185C332F186C333F1010127
:102A4000296B55EC3CF0CCEC3BF003018351300A90
:102A5000D8B439EF15F003018351310AD8B441EFEE
:102A600015F003018351320AD8B449EF15F01DEF78
:102A700034F0FD0E0C6E00C10BF0F1EC0BF051EFD9
:102A800015F0FE0E0C6E00C10BF0F1EC0BF064EFD4
:102A900015F0FF0E0C6E00C10BF0F1EC0BF077EFB0
:102AA00015F00401300E826F70EC0FF004012C0E53
:102AB000826F70EC0FF007EC3CF0FD0E08EC0CF0B0
:102AC000E8CF00F188EF15F00401310E826F70EC51
:102AD0000FF004012C0E826F70EC0FF007EC3CF04D
:102AE000FE0E08EC0CF0E8CF00F188EF15F00401C1
:102AF000320E826F70EC0FF007EC3CF004012C0EEC
:102B0000826F70EC0FF0FF0E08EC0CF0E8CF00F1D4
:102B100090EC3BF031C182F40401300E822770EC5E
:102B20000FF032C182F40401300E822770EC0FF0F6
:102B300033C182F40401300E822770EC0FF01BEFDA
:102B400034F003018351300AD8B446EF17F0030183
:102B50008351310AD8B47DEF17F003018351320A53
:102B6000D8B432EF19F003018351330AD8B4E7EF38
:102B70001AF003018351340AD8B48DEF1BF003011E
:102B80008351730AD8B428EF16F003018351760AF3
:102B9000D8B42AEF16F003018351740AD8B415EFA4
:102BA00016F003018351540AD8B4DAEF15F0D8A413
:102BB0001DEF34F00401760E826F70EC0FF004010B
:102BC000540E826F70EC0FF007840001880E0C6EBB
:102BD00048EC3CF02981030184512D0AD8B4F3EF6D
:102BE00015F00101299185C32FF186C330F187C308
:102BF00031F188C332F189C333F155EC3CF0CCECB0
:102C00003BF000C10BF0F1EC0BF001C10BF0F1EC6B
:102C10000BF0880E08EC0CF0E8CF40F6890E08ECBB
:102C20000CF0E8CF41F620EF16F00401760E826F2B
:102C300070EC0FF00401740E826F70EC0FF00784DB
:102C40000001880E0C6E0FEC0CF00794D4EF27F007
:102C500028EC16F00401760E826F70EC0FF0040180
:102C6000760E826F70EC0FF007844AEC38F00401A6
:102C70002C0E826F70EC0FF00101036B026B3BC6F0
:102C800001F13AC600F101AF4BEF16F00101FF0E62
:102C9000026FFF0E036F90EC3BF0296752EF16F0C6
:102CA00057EF16F004012D0E826F70EC0FF02FC15C
:102CB00082F40401300E822770EC0FF030C182F4F0
:102CC0000401300E822770EC0FF031C182F4040150
:102CD000300E822770EC0FF032C182F40401300E06
:102CE000822770EC0FF033C182F40401300E82278A
:102CF00070EC0FF004012C0E826F70EC0FF00101EC
:102D0000036B026B3DC601F13CC600F101AF8EEFD3
:102D100016F00101FF0E026FFF0E036F90EC3BF007
:102D2000296795EF16F09AEF16F004012D0E826FC9
:102D300070EC0FF02FC182F40401300E822770EC8A
:102D40000FF030C182F40401300E822770EC0FF0D6
:102D500031C182F40401300E822770EC0FF032C1D1
:102D600082F40401300E822770EC0FF033C182F43C
:102D70000401300E822770EC0FF004012C0E826FDC
:102D800070EC0FF00101036B026B3FC601F13EC610
:102D900000F101AFD1EF16F00101FF0E026FFF0E3F
:102DA000036F90EC3BF02967D8EF16F0DDEF16F0DB
:102DB00004012D0E826F70EC0FF02FC182F404011C
:102DC000300E822770EC0FF030C182F40401300E17
:102DD000822770EC0FF031C182F40401300E82279B
:102DE00070EC0FF032C182F40401300E822770ECD7
:102DF0000FF033C182F40401300E822770EC0FF023
:102E000004012C0E826F70EC0FF00101036B026B5A
:102E100037C601F136C600F101AF14EF17F001011A
:102E2000FF0E026FFF0E036F90EC3BF029671BEF64
:102E300017F020EF17F004012D0E826F70EC0FF0E9
:102E40002FC182F40401300E822770EC0FF030C1E4
:102E500082F40401300E822770EC0FF031C182F44D
:102E60000401300E822770EC0FF032C182F40401AD
:102E7000300E822770EC0FF033C182F40401300E63
:102E8000822770EC0FF00794D4EF27F00401760E40
:102E9000826F70EC0FF00401300E826F70EC0FF057
:102EA00004012C0E826F70EC0FF08EEC3CF007ECFE
:102EB0003CF000C600F101C601F190EC3BF030C1DE
:102EC00082F40401300E822770EC0FF031C182F4DD
:102ED0000401300E822770EC0FF032C182F404013D
:102EE000300E822770EC0FF033C182F40401300EF3
:102EF000822770EC0FF0D4EF27F00401760E826F7A
:102F000070EC0FF00401310E826F70EC0FF007844B
:102F10000101036B026B02C600F103C601F101AFB0
:102F200096EF17F0FF0E026FFF0E036F0101076BA4
:102F3000066B04C604F105C605F105AFA4EF17F052
:102F4000FF0E066FFF0E076FF7EC3AF00101076BFB
:102F5000066B06C604F107C605F105AFB4EF17F01E
:102F6000FF0E066FFF0E076FF7EC3AF00101076BDB
:102F7000066B08C604F109C605F105AFC4EF17F0EA
:102F8000FF0E066FFF0E076FF7EC3AF0D8900101C5
:102F90000333023301330033D8900101033302338A
:102FA0000133003304012C0E826F70EC0FF001012D
:102FB000036B026B01C101F100C100F101AFE6EF4B
:102FC00017F00101FF0E026FFF0E036F90EC3BF054
:102FD0002967EDEF17F0F2EF17F004012D0E826F65
:102FE00070EC0FF02FC182F40401300E822770ECD8
:102FF0000FF030C182F40401300E822770EC0FF024
:1030000031C182F40401300E822770EC0FF032C11E
:1030100082F40401300E822770EC0FF033C182F489
:103020000401300E822770EC0FF00101036B026B7C
:103030000AC600F10BC601F101AF23EF18F0FF0E35
:10304000026FFF0E036F0101076B066B0CC604F1E4
:103050000DC605F105AF31EF18F0FF0E066FFF0E3C
:10306000076FF7EC3AF00101076B066B0EC604F12F
:103070000FC605F105AF41EF18F0FF0E066FFF0E0A
:10308000076FF7EC3AF00101076B066B10C604F10D
:1030900011C605F105AF51EF18F0FF0E066FFF0ED8
:1030A000076FF7EC3AF0D890010103330233013394
:1030B0000033D8900101033302330133003304019C
:1030C0002C0E826F70EC0FF00101036B026B01C1DB
:1030D00001F100C100F101AF73EF18F00101FF0E23
:1030E000026FFF0E036F90EC3BF029677AEF18F048
:1030F0007FEF18F004012D0E826F70EC0FF02FC1DE
:1031000082F40401300E822770EC0FF030C182F49B
:103110000401300E822770EC0FF031C182F40401FB
:10312000300E822770EC0FF032C182F40401300EB1
:10313000822770EC0FF033C182F40401300E822735
:1031400070EC0FF00101036B026B12C600F113C6A5
:1031500001F101AFB0EF18F0FF0E026FFF0E036F29
:103160000101076B066B14C604F115C605F105AF26
:10317000BEEF18F0FF0E066FFF0E076FF7EC3AF088
:103180000101076B066B16C604F117C605F105AF02
:10319000CEEF18F0FF0E066FFF0E076FF7EC3AF058
:1031A0000101076B066B18C604F119C605F105AFDE
:1031B000DEEF18F0FF0E066FFF0E076FF7EC3AF028
:1031C000D89001010333023301330033D890010159
:1031D000033302330133003304012C0E826F70EC91
:1031E0000FF00101036B026B01C101F100C100F19D
:1031F00001AF00EF19F00101FF0E026FFF0E036F28
:1032000090EC3BF0296707EF19F00CEF19F004017F
:103210002D0E826F70EC0FF02FC182F40401300E7E
:10322000822770EC0FF030C182F40401300E822747
:1032300070EC0FF031C182F40401300E822770EC83
:103240000FF032C182F40401300E822770EC0FF0CF
:1032500033C182F40401300E822770EC0FF0079422
:10326000D4EF27F00401760E826F70EC0FF00401AA
:10327000320E826F70EC0FF007840101036B026B5A
:103280001AC600F11BC601F101AF4BEF19F0FF0E9A
:10329000026FFF0E036F0101076B066B1CC604F182
:1032A0001DC605F105AF59EF19F0FF0E066FFF0EB1
:1032B000076FF7EC3AF00101076B066B1EC604F1CD
:1032C0001FC605F105AF69EF19F0FF0E066FFF0E7F
:1032D000076FF7EC3AF00101076B066B20C604F1AB
:1032E00021C605F105AF79EF19F0FF0E066FFF0E4D
:1032F000076FF7EC3AF0D890010103330233013342
:103300000033D89001010333023301330033040149
:103310002C0E826F70EC0FF00101036B026B01C188
:1033200001F100C100F101AF9BEF19F00101FF0EA7
:10333000026FFF0E036F90EC3BF02967A2EF19F0CC
:10334000A7EF19F004012D0E826F70EC0FF02FC162
:1033500082F40401300E822770EC0FF030C182F449
:103360000401300E822770EC0FF031C182F40401A9
:10337000300E822770EC0FF032C182F40401300E5F
:10338000822770EC0FF033C182F40401300E8227E3
:1033900070EC0FF00101036B026B22C600F123C633
:1033A00001F101AFD8EF19F0FF0E026FFF0E036FAE
:1033B0000101076B066B24C604F125C605F105AFB4
:1033C000E6EF19F0FF0E066FFF0E076FF7EC3AF00D
:1033D0000101076B066B26C604F127C605F105AF90
:1033E000F6EF19F0FF0E066FFF0E076FF7EC3AF0DD
:1033F0000101076B066B28C604F129C605F105AF6C
:1034000006EF1AF0FF0E066FFF0E076FF7EC3AF0AB
:10341000D89001010333023301330033D890010106
:10342000033302330133003304012C0E826F70EC3E
:103430000FF00101036B026B01C101F100C100F14A
:1034400001AF28EF1AF00101FF0E026FFF0E036FAC
:1034500090EC3BF029672FEF1AF034EF1AF00401DB
:103460002D0E826F70EC0FF02FC182F40401300E2C
:10347000822770EC0FF030C182F40401300E8227F5
:1034800070EC0FF031C182F40401300E822770EC31
:103490000FF032C182F40401300E822770EC0FF07D
:1034A00033C182F40401300E822770EC0FF0010169
:1034B000036B026B2AC600F12BC601F101AF65EF69
:1034C0001AF0FF0E026FFF0E036F0101076B066B10
:1034D0002CC604F12DC605F105AF73EF1AF0FF0EEF
:1034E000066FFF0E076FF7EC3AF00101076B066BF2
:1034F0002EC604F12FC605F105AF83EF1AF0FF0EBB
:10350000066FFF0E076FF7EC3AF00101076B066BD1
:1035100030C604F131C605F105AF93EF1AF0FF0E86
:10352000066FFF0E076FF7EC3AF0D89001010333F6
:10353000023301330033D8900101033302330133E6
:10354000003304012C0E826F70EC0FF00101036B4D
:10355000026B01C101F100C100F101AFB5EF1AF03A
:103560000101FF0E026FFF0E036F90EC3BF0296725
:10357000BCEF1AF0C1EF1AF004012D0E826F70EC4F
:103580000FF02FC182F40401300E822770EC0FF08F
:1035900030C182F40401300E822770EC0FF031C18B
:1035A00082F40401300E822770EC0FF032C182F4F5
:1035B0000401300E822770EC0FF033C182F4040155
:1035C000300E822770EC0FF00794D4EF27F004013F
:1035D000760E826F70EC0FF00401330E826F70EC88
:1035E0000FF004012C0E826F70EC0FF085C382F493
:1035F00070EC0FF0640E0D6E03018551320A02E18A
:103600006A0E0D6E03018551330A02E1700E0D6ED4
:1036100003018551340A02E1760E0D6E03018551D6
:10362000350A02E17C0E0D6E03018551360A02E176
:10363000820E0D6E03018651780A65E00DC00CF014
:1036400048EC3CF02981030187512D0AD8B42BEFB7
:103650001BF00101299188C32FF189C330F18AC37E
:1036600031F18BC332F18CC333F155EC3CF0CCEC2F
:103670003BF000C10BF0F1EC0BF001C10BF0F1ECF1
:103680000BF048EC3CF0298103018E512D0AD8B48F
:103690004CEF1BF0010129918FC32FF190C330F142
:1036A00091C331F192C332F193C333F155EC3CF045
:1036B000CCEC3BF000C10BF0F1EC0BF001C10BF0D6
:1036C000F1EC0BF048EC3CF02981030195512D0AF7
:1036D000D8B46DEF1BF00101299196C32FF197C368
:1036E00030F198C331F199C332F19AC333F155ECFB
:1036F0003CF0CCEC3BF000C10BF0F1EC0BF001C165
:103700000BF0F1EC0BF00DC00CF00FEC0CF00FEC2B
:103710000CF00FEC0CF0D4EF27F00401760E826F62
:1037200070EC0FF00401340E826F70EC0FF00301A7
:103730008451780AD8B465EF1CF03E0E0C6E48EC4C
:103740003CF02981030185512D0AD8B4AAEF1BF062
:103750000101299186C32FF187C330F188C331F16C
:1037600089C332F18AC333F155EC3CF0CCEC3BF029
:1037700000C10BF0F1EC0BF001C10BF0F1EC0BF020
:1037800048EC3CF0298103018C512D0AD8B4CBEFD1
:103790001BF0010129918DC32FF18EC330F18FC32E
:1037A00031F190C332F191C333F155EC3CF0CCECE4
:1037B0003BF000C10BF0F1EC0BF001C10BF0F1ECB0
:1037C0000BF048EC3CF02981030193512D0AD8B449
:1037D000ECEF1BF00101299194C32FF195C330F157
:1037E00096C331F197C332F198C333F155EC3CF0F5
:1037F000CCEC3BF000C10BF0F1EC0BF001C10BF095
:10380000F1EC0BF048EC3CF0298103019A512D0AB0
:10381000D8B40DEF1CF0010129919BC32FF19CC37B
:1038200030F19DC331F19EC332F19FC333F155ECAA
:103830003CF0CCEC3BF000C10BF0F1EC0BF001C123
:103840000BF0F1EC0BF048EC3CF029810301A151A5
:103850002D0AD8B42EEF1CF001012991A2C32FF13B
:10386000A3C330F1A4C331F1A5C332F1A6C333F130
:1038700055EC3CF0CCEC3BF000C10BF0F1EC0BF064
:1038800001C10BF0F1EC0BF048EC3CF02981030195
:10389000A8512D0AD8B44FEF1CF001012991A9C3FA
:1038A0002FF1AAC330F1ABC331F1ACC332F1ADC3D8
:1038B00033F155EC3CF0CCEC3BF000C10BF0F1ECFB
:1038C0000BF001C10BF0F1EC0BF03E0E0C6E0FECA7
:1038D0000CF00FEC0CF00FEC0CF00FEC0CF00FEC0C
:1038E0000CF00FEC0CF0D4EF27F003018351300AF9
:1038F000D8B4C9EF21F003018351310AD8B4F6EFEF
:1039000022F003018351320AD8B464EF23F003019B
:103910008351330AD8B474EF23F003018351340A7E
:10392000D8B4CFEF23F003018351350AD8B478EF30
:1039300027F003018351360AD8B4A6EF27F003011C
:103940008351370AD8B4A1EF1FF003018351380A1D
:10395000D8B43FEF20F003018351440AD8B4CDEF2F
:103960001DF003018351640AD8B4EDEF1DF003018B
:103970008351460AD8B47DEF26F0030183514D0AE6
:10398000D8B41AEF1EF0030183516D0AD8B434EF96
:103990001EF0030183515A0AD8B470EF22F00301DC
:1039A0008351490AD8B4A6EF28F003018351500A85
:1039B000D8B4D8EF27F003018351540AD8B451EF9B
:1039C00028F003018351630AD8B454EF1EF00301B9
:1039D0008351430AD8B44CEF1FF003018351730A9B
:1039E000D8B452EF1EF003018351610AD8B41AEF24
:1039F0001DF003018351650AD8B419EF22F00301C9
:103A00008351450AD8B427EF22F003018351620A9B
:103A1000D8B435EF22F003018351420AD8B443EF02
:103A200022F003018351760AD8B451EF22F0D8A4D2
:103A30001DEF34F004014C0E826F70EC0FF00401A6
:103A4000610E826F70EC0FF088EC3EF004012C0EDA
:103A5000826F70EC0FF007EC3CF0AFC500F1010194
:103A600090EC3BF031C182F40401300E822770ECFF
:103A70000FF032C182F40401300E822770EC0FF097
:103A800033C182F40401300E822770EC0FF0040180
:103A90002C0E826F70EC0FF007EC3CF0B0C500F11B
:103AA000010190EC3BF031C182F40401300E822719
:103AB00070EC0FF032C182F40401300E822770ECFA
:103AC0000FF033C182F40401300E822770EC0FF046
:103AD00004012C0E826F70EC0FF007EC3CF0B1C5C6
:103AE00000F1010190EC3BF031C182F40401300E91
:103AF000822770EC0FF032C182F40401300E82276D
:103B000070EC0FF033C182F40401300E822770ECA8
:103B10000FF004012C0E826F70EC0FF007EC3CF0FC
:103B2000B2C500F1010190EC3BF031C182F4040117
:103B3000300E822770EC0FF032C182F40401300E97
:103B4000822770EC0FF033C182F40401300E82271B
:103B500070EC0FF004012C0E826F70EC0FF007EC8C
:103B60003CF0B6C500F1010190EC3BF031C182F4AC
:103B70000401300E822770EC0FF032C182F4040190
:103B8000300E822770EC0FF033C182F40401300E46
:103B9000822770EC0FF0D4EF27F003018451300A34
:103BA000D8B4D9EF1DF003018451310AD8B4DDEF48
:103BB0001DF015921596DEEF1DF01582C70E08EC6C
:103BC0000CF0E8CF00F10101008115A20091C70EB1
:103BD0000C6E00C10BF0F1EC0BF0C70E08EC0CF012
:103BE000E8CF00F1010100B1F9EF1DF01592FAEFF5
:103BF0001DF0158204014C0E826F70EC0FF0040171
:103C0000640E826F70EC0FF004012C0E826F70EC6A
:103C10000FF015B213EF1EF00401300E826F70EC3E
:103C20000FF018EF1EF00401310E826F70EC0FF0F0
:103C30001BEF34F048EC3CF084C333F155EC3CF01E
:103C4000CCEC3BF0200E0C6E00C10BF0F1EC0BF055
:103C500000C12FF505012F51000A06E005012F5183
:103C6000010A02E022EC3FF004014C0E826F70EC7E
:103C70000FF004014D0E826F70EC0FF004012C0E5A
:103C8000826F70EC0FF007EC3CF02FC500F190EC68
:103C90003BF033C182F40401300E822770EC0FF048
:103CA000D4EF27F000EF47F004014C0E826F70EC68
:103CB0000FF00401630E826F70EC0FF0E0EC3DF04A
:103CC00004012C0E826F70EC0FF069EC1EF0D4EF43
:103CD00027F007EC3CF0B5C500F10101003B0F0EE9
:103CE000001790EC3BF033C182F40401300E8227C0
:103CF00070EC0FF0B5C500F101010F0E01010017C6
:103D000090EC3BF033C182F40401300E822770EC5A
:103D10000FF004012D0E826F70EC0FF0B4C500F1AE
:103D20000101003B0F0E001790EC3BF033C182F411
:103D30000401300E822770EC0FF0B4C500F10101D0
:103D40000F0E0101001790EC3BF033C182F4040127
:103D5000300E822770EC0FF004012D0E826F70EC94
:103D60000FF0B3C500F10101003B0F0E001790ECFE
:103D70003BF033C182F40401300E822770EC0FF067
:103D8000B3C500F101010F0E0101001790EC3BF0EB
:103D900033C182F40401300E822770EC0FF004016D
:103DA000200E826F70EC0FF0B2C500F10F0E010112
:103DB000001790EC3BF033C182F40401300E8227EF
:103DC00070EC0FF00401200E826F70EC0FF0B1C5A3
:103DD00000F101010101003B0F0E001790EC3BF0D8
:103DE00033C182F40401300E822770EC0FF0B1C5AC
:103DF00000F101010F0E0101001790EC3BF033C1FF
:103E000082F40401300E822770EC0FF004013A0EA8
:103E1000826F70EC0FF0B0C500F10101003B0F0E96
:103E2000001790EC3BF033C182F40401300E82277E
:103E300070EC0FF0B0C500F101010F0E0101001789
:103E400090EC3BF033C182F40401300E822770EC19
:103E50000FF004013A0E826F70EC0FF0AFC500F165
:103E60000101003B0F0E001790EC3BF033C182F4D0
:103E70000401300E822770EC0FF0AFC500F1010194
:103E80000F0E001790EC3BF033C182F40401300EAA
:103E9000822770EC0FF0120084C3E8FF0F0BE83AA2
:103EA000E8CFB5F585C3E8FF0F0B0501B51387C350
:103EB000E8FF0F0BE83AE8CFB4F588C3E8FF0F0B33
:103EC0000501B4138AC3E8FF0F0BE83AE8CFB3F556
:103ED0008BC3E8FF0F0B0501B3138DC3E8FF0F0B76
:103EE000E8CFB2F58FC3E8FF0F0BE83AE8CFB1F5A2
:103EF00090C3E8FF0F0B0501B11392C3E8FF0F0B4E
:103F0000E83AE8CFB0F593C3E8FF0F0B0501B01313
:103F100095C3E8FF0F0BE83AE8CFAFF596C3E8FF8B
:103F20000F0B0501AF133BEC3EF004014C0E826F0A
:103F300070EC0FF00401430E826F70EC0FF05EEF37
:103F40001EF0078404014C0E826F70EC0FF0040128
:103F5000370E826F70EC0FF004012C0E826F70EC44
:103F60000FF005012E51130A06E005012E51170A24
:103F70000DE03CEF20F00101000E006F000E016F1C
:103F8000100E026F000E036FCFEF1FF00101000E45
:103F9000006F000E016F000E026F010E036F90ECB8
:103FA0003BF02AC182F40401300E822770EC0FF03E
:103FB0002BC182F40401300E822770EC0FF02CC16B
:103FC00082F40401300E822770EC0FF02DC182F4D0
:103FD0000401300E822770EC0FF02EC182F4040130
:103FE000300E822770EC0FF02FC182F40401300EE6
:103FF000822770EC0FF030C182F40401300E82276A
:1040000070EC0FF031C182F40401300E822770ECA5
:104010000FF032C182F40401300E822770EC0FF0F1
:1040200033C182F40401300E822770EC0FF00401DA
:104030002C0E826F70EC0FF00101200E006F000E4D
:10404000016F000E026F000E036F90EC3BF031C168
:1040500082F40401300E822770EC0FF032C182F43A
:104060000401300E822770EC0FF033C182F404019A
:10407000300E822770EC0FF00794D4EF27F0050183
:10408000216B226B236B246B04014C0E826F70EC4E
:104090000FF00401380E826F70EC0FF004012C0E4B
:1040A000826F70EC0FF00101200E006F000E016FA7
:1040B000000E026F000E036F90EC3BF02AC182F4F9
:1040C0000401300E822770EC0FF02BC182F4040142
:1040D000300E822770EC0FF02CC182F40401300EF8
:1040E000822770EC0FF02DC182F40401300E82277C
:1040F00070EC0FF02EC182F40401300E822770ECB8
:104100000FF02FC182F40401300E822770EC0FF003
:1041100030C182F40401300E822770EC0FF031C1FF
:1041200082F40401300E822770EC0FF032C182F469
:104130000401300E822770EC0FF033C182F40401C9
:10414000300E822770EC0FF004012C0E826F70ECA1
:104150000FF025C500F126C501F127C502F128C5DC
:1041600003F10101200E046F000E056F000E066FB3
:10417000000E076F23EC3BF000C133F501C134F5AD
:1041800002C135F503C136F590EC3BF02AC182F44B
:104190000401300E822770EC0FF02BC182F4040171
:1041A000300E822770EC0FF02CC182F40401300E27
:1041B000822770EC0FF02DC182F40401300E8227AB
:1041C00070EC0FF02EC182F40401300E822770ECE7
:1041D0000FF02FC182F40401300E822770EC0FF033
:1041E00030C182F40401300E822770EC0FF031C12F
:1041F00082F40401300E822770EC0FF032C182F499
:104200000401300E822770EC0FF033C182F40401F8
:10421000300E822770EC0FF07AEC0FF00501336757
:1042200019EF21F0346719EF21F0356719EF21F00C
:10423000366702D0B8EF21F0129E129C21C500F122
:1042400022C501F123C502F124C503F1899A400E6C
:10425000C76E200EC66E9E96C69E0B0EC96EFF0ED2
:104260009EB602D0E82EFCD79E96C69E02C1C9FF1C
:10427000FF0E9EB602D0E82EFCD79E96C69E01C1C8
:10428000C9FFFF0E9EB602D0E82EFCD79E96C69EB2
:1042900000C1C9FFFF0E9EB602D0E82EFCD79E9645
:1042A000C69EC952FF0E9EB602D0E82EFCD705016D
:1042B000200E326F040114EE00F080517F0BE126D6
:1042C0009E96C69EC952FF0E9EB602D0E82EFCD71F
:1042D000C9CFE7FF0401802B0501322F5AEF21F0EF
:1042E000898A33C500F134C501F135C502F136C5FF
:1042F00003F10101010E046F000E056F000E066F41
:10430000000E076FF2EC3AF000C133F501C134F54D
:1043100002C135F503C136F50501336797EF21F08A
:10432000346797EF21F0356797EF21F0366702D0B9
:10433000B8EF21F021C500F122C501F123C502F13A
:1043400024C503F10101200E046F000E056F000E5D
:10435000066F000E076FF7EC3AF000C121F501C1BE
:1043600022F502C123F503C124F5128E1DEF34F0AE
:104370000401450E826F70EC0FF004014F0E826F46
:1043800070EC0FF00401460E826F70EC0FF0D4EF6A
:1043900027F007845AEC46F007EC3CF02DC500F1FD
:1043A00090EC3BF004014C0E826F70EC0FF00401B6
:1043B000300E826F70EC0FF004012C0E826F70ECE7
:1043C0000FF031C182F40401300E822770EC0FF03F
:1043D00032C182F40401300E822770EC0FF033C139
:1043E00082F40401300E822770EC0FF004012C0ED1
:1043F000826F70EC0FF007EC3CF02EC500F190ECF2
:104400003BF031C182F40401300E822770EC0FF0D2
:1044100032C182F40401300E822770EC0FF033C1F8
:1044200082F40401300E822770EC0FF00794D4EF71
:1044300027F004014C0E826F70EC0FF00401650E42
:10444000826F70EC0FF0FEEC3FF0D4EF27F0040128
:104450004C0E826F70EC0FF00401450E826F70EC11
:104460000FF015EC40F0D4EF27F004014C0E826FF2
:1044700070EC0FF00401620E826F70EC0FF043ECF1
:1044800040F0D4EF27F004014C0E826F70EC0FF077
:104490000401420E826F70EC0FF02CEC40F0D4EF70
:1044A00027F004014C0E826F70EC0FF00401760EC1
:1044B000826F70EC0FF004012C0E826F70EC0FF025
:1044C00010A807D00401310E826F70EC0FF0D4EF0A
:1044D00027F00401300E826F70EC0FF0D4EF27F05C
:1044E00004014C0E826F70EC0FF004015A0E826FC3
:1044F00070EC0FF004012C0E826F70EC0FF05AEC90
:1045000046F007EC3CF005012E51130A06E00501C8
:104510002E51170A0DE0A1EF22F00101000E006FED
:10452000000E016F100E026F000E036FA1EF22F05C
:104530000101000E006F000E016F000E026F010EF0
:10454000036F0101200E046F000E056F000E066F51
:10455000000E076F23EC3BF090EC3BF02AC182F495
:104560000401300E822770EC0FF02BC182F404019D
:10457000300E822770EC0FF02CC182F40401300E53
:10458000822770EC0FF02DC182F40401300E8227D7
:1045900070EC0FF02EC182F40401300E822770EC13
:1045A0000FF02FC182F40401300E822770EC0FF05F
:1045B00030C182F40401300E822770EC0FF031C15B
:1045C00082F40401300E822770EC0FF032C182F4C5
:1045D0000401300E822770EC0FF033C182F4040125
:1045E000300E822770EC0FF0D4EF27F0078404011F
:1045F0004C0E826F70EC0FF00401310E826F70EC84
:104600000FF004012C0E826F70EC0FF025C500F145
:1046100026C501F127C502F128C503F10101200ECD
:10462000046F000E056F000E066F000E076F23EC7F
:104630003BF090EC3BF02AC182F40401300E82275B
:1046400070EC0FF02BC182F40401300E822770EC65
:104650000FF02CC182F40401300E822770EC0FF0B1
:104660002DC182F40401300E822770EC0FF02EC1B0
:1046700082F40401300E822770EC0FF02FC182F417
:104680000401300E822770EC0FF030C182F4040177
:10469000300E822770EC0FF031C182F40401300E2D
:1046A000822770EC0FF032C182F40401300E8227B1
:1046B00070EC0FF033C182F40401300E822770ECED
:1046C0000FF00794D4EF27F0078404014C0E826F9B
:1046D00070EC0FF00401320E826F70EC0FF032ECD0
:1046E00042F00794D4EF27F0078437B07AEF23F035
:1046F0008DEF23F0010E166E04014C0E826F70ECEC
:104700000FF00401330E826F70EC0FF08FEC42F06B
:10471000000E166E079401EF23F0020E166E8FEC5A
:1047200042F08B800501010E306F3C0E316F0101AC
:104730005E6B5F6B606B616B626B636B646B656B15
:10474000666B676B686B696B536B546BCF6ACE6A31
:104750000F9A0F9C0F9E030E166E04014C0E826F73
:1047600070EC0FF00401330E826F70EC0FF0040157
:104770002C0E826F70EC0FF004012D0E826F70EC26
:104780000FF00401310E826F70EC0FF01BEF34F06C
:104790008FEC42F0000E166E8B901DEF34F0078404
:1047A00004014C0E826F70EC0FF00401340E826F26
:1047B00070EC0FF004012C0E826F70EC0FF048ECDF
:1047C0003CF084C32AF185C32BF186C32CF187C347
:1047D0002DF188C32EF189C32FF18AC330F18BC329
:1047E00031F18CC332F18DC333F10101296B55ECEA
:1047F0003CF0CCEC3BF0200E046F000E056F000E79
:10480000066F000E076F03EC3BF000C121F501C1FC
:1048100022F502C123F503C124F50DEC46F038C59D
:10482000AFF539C5B0F53AC5B1F53BC5B2F53CC5F4
:10483000B3F53DC5B4F53EC5B5F569EC1EF0040110
:104840002C0E826F70EC0FF03FC500F140C501F1F6
:1048500041C502F142C503F10101000E046F000ED3
:10486000056F010E066F000E076F23EC3BF090EC16
:104870003BF029673EEF24F043EF24F004012D0EB6
:10488000826F70EC0FF030C182F40401300E822789
:1048900070EC0FF031C182F40401300E822770EC0D
:1048A0000FF004012E0E826F70EC0FF032C182F413
:1048B0000401300E822770EC0FF033C182F4040142
:1048C000300E822770EC0FF004012C0E826F70EC1A
:1048D0000FF007EC3CF043C500F144C501F147EC93
:1048E00035F004012C0E826F70EC0FF007EC3CF0F9
:1048F00045C500F190EC3BF031C182F40401300E6B
:10490000822770EC0FF032C182F40401300E82274E
:1049100070EC0FF033C182F40401300E822770EC8A
:104920000FF004012C0E826F70EC0FF00101036B8D
:10493000026B4CC501F14BC500F101AFA5EF24F0AE
:104940000101FF0E026FFF0E036F90EC3BF0296731
:10495000ACEF24F0B1EF24F004012D0E826F70EC67
:104960000FF02FC182F40401300E822770EC0FF09B
:1049700030C182F40401300E822770EC0FF031C197
:1049800082F40401300E822770EC0FF032C182F401
:104990000401300E822770EC0FF033C182F4040161
:1049A000300E822770EC0FF004012C0E826F70EC39
:1049B0000FF00101036B026B4EC501F14DC500F113
:1049C00001AFE8EF24F00101FF0E026FFF0E036F4D
:1049D00090EC3BF02967EFEF24F0F4EF24F00401B2
:1049E0002D0E826F70EC0FF02FC182F40401300E97
:1049F000822770EC0FF030C182F40401300E822760
:104A000070EC0FF031C182F40401300E822770EC9B
:104A10000FF032C182F40401300E822770EC0FF0E7
:104A200033C182F40401300E822770EC0FF00401D0
:104A30002C0E826F70EC0FF00101036B026B50C5FE
:104A400001F14FC500F101AF2BEF25F00101FF0E81
:104A5000026FFF0E036F90EC3BF0296732EF25F0F9
:104A600037EF25F004012D0E826F70EC0FF02FC18F
:104A700082F40401300E822770EC0FF030C182F412
:104A80000401300E822770EC0FF031C182F4040172
:104A9000300E822770EC0FF032C182F40401300E28
:104AA000822770EC0FF033C182F40401300E8227AC
:104AB00070EC0FF004012C0E826F70EC0FF001010E
:104AC000036B026B52C501F151C500F101AF6EEFEE
:104AD00025F00101FF0E026FFF0E036F90EC3BF01B
:104AE000296775EF25F07AEF25F004012D0E826F0E
:104AF00070EC0FF02FC182F40401300E822770ECAD
:104B00000FF030C182F40401300E822770EC0FF0F8
:104B100031C182F40401300E822770EC0FF032C1F3
:104B200082F40401300E822770EC0FF033C182F45E
:104B30000401300E822770EC0FF004012C0E826FFE
:104B400070EC0FF00101036B026B54C501F153C50A
:104B500000F101AFB1EF25F00101FF0E026FFF0E72
:104B6000036F90EC3BF02967B8EF25F0BDEF25F01F
:104B700004012D0E826F70EC0FF02FC182F404013E
:104B8000300E822770EC0FF030C182F40401300E39
:104B9000822770EC0FF031C182F40401300E8227BD
:104BA00070EC0FF032C182F40401300E822770ECF9
:104BB0000FF033C182F40401300E822770EC0FF045
:104BC00004012C0E826F70EC0FF00101036B026B7D
:104BD00056C501F155C500F101AFF4EF25F0010113
:104BE000FF0E026FFF0E036F90EC3BF02967FBEFA7
:104BF00025F000EF26F004012D0E826F70EC0FF00F
:104C00002FC182F40401300E822770EC0FF030C106
:104C100082F40401300E822770EC0FF031C182F46F
:104C20000401300E822770EC0FF032C182F40401CF
:104C3000300E822770EC0FF033C182F40401300E85
:104C4000822770EC0FF004012C0E826F70EC0FF0D5
:104C50000101036B026B4AC501F149C500F101AFC7
:104C600037EF26F00101FF0E026FFF0E036F90EC8D
:104C70003BF029673EEF26F043EF26F004012D0EAE
:104C8000826F70EC0FF02FC182F40401300E822786
:104C900070EC0FF030C182F40401300E822770EC0A
:104CA0000FF031C182F40401300E822770EC0FF056
:104CB00032C182F40401300E822770EC0FF033C150
:104CC00082F40401300E822770EC0FF004012C0EE8
:104CD000826F70EC0FF037C5E8FFE8B806D004012A
:104CE000300E826F70EC0FF005D00401310E826F30
:104CF00070EC0FF00794D4EF27F048EC3CF085C33C
:104D00002AF186C32BF187C32CF188C32DF189C307
:104D10002EF18AC32FF18BC330F18CC331F18DC3D7
:104D200032F18EC333F10101296B55EC3CF0CCEC30
:104D30003BF00101010E046F000E056F000E066FBF
:104D4000000E076FF2EC3AF0100E046F000E056FC4
:104D5000000E066F000E076F03EC3BF000C129F553
:104D600001C12AF502C12BF503C12CF5B9EC41F0C4
:104D700004014C0E826F70EC0FF00401460E826F3E
:104D800070EC0FF004012C0E826F70EC0FF025C553
:104D900000F126C501F127C502F128C503F1010183
:104DA000100E046F000E056F000E066F000E076FE9
:104DB00023EC3BF090EC3BF02AC182F40401300E6E
:104DC000822770EC0FF02BC182F40401300E822791
:104DD00070EC0FF02CC182F40401300E822770ECCD
:104DE0000FF02DC182F40401300E822770EC0FF019
:104DF0002EC182F40401300E822770EC0FF02FC117
:104E000082F40401300E822770EC0FF030C182F47E
:104E10000401300E822770EC0FF031C182F40401DE
:104E2000300E822770EC0FF032C182F40401300E94
:104E3000822770EC0FF033C182F40401300E822718
:104E400070EC0FF0D4EF27F037B029EF27F0020E07
:104E5000166E8FEC42F000011650020AD8B447EFEC
:104E600027F005012F51010AD8B43DEF27F015B204
:104E700042EF27F081BA42EF27F0000E166E15843C
:104E80001DEF34F0050E166E158400EF47F08B8091
:104E900001015E6B5F6B606B616B626B636B646B7C
:104EA000656B666B676B686B696B536B546BCF6A32
:104EB000CE6A0F9A0F9C0F9E030E166E1DEF34F0F4
:104EC0008FEC42F005012F51010AD8B46EEF27F0A4
:104ED00015B273EF27F081BA73EF27F0000E166E4C
:104EE00015841DEF34F0050E166E158400EF47F0A3
:104EF00004014C0E826F70EC0FF00401350E826FCE
:104F000070EC0FF004012C0E826F70EC0FF007ECC8
:104F10003CF00784B9C500F1079490EC3BF031C137
:104F200082F40401300E822770EC0FF032C182F45B
:104F30000401300E822770EC0FF033C182F40401BB
:104F4000300E822770EC0FF0D4EF27F052EC42F0D5
:104F500007EC3CF037C500F190EC3BF004014C0E3F
:104F6000826F70EC0FF00401360E826F70EC0FF060
:104F700004012C0E826F70EC0FF031C182F4040139
:104F8000300E822770EC0FF032C182F40401300E33
:104F9000822770EC0FF033C182F40401300E8227B7
:104FA00070EC0FF0D4EF27F07AEC0FF01DEF34F037
:104FB00004014C0E826F70EC0FF00401500E826FF2
:104FC00070EC0FF004012C0E826F70EC0FF085C3B3
:104FD0002AF186C32BF187C32CF188C32DF189C335
:104FE0002EF18AC32FF18BC330F18CC331F18DC305
:104FF00032F18EC333F1010155EC3CF0CCEC3BF0C7
:1050000003018451530A0DE0030184514D0A38E035
:105010000401780E826F70EC0FF07AEC0FF01DEF48
:1050200034F00401530E826F70EC0FF0250E0C6EFD
:1050300000C10BF0F1EC0BF0260E0C6E01C10BF071
:10504000F1EC0BF0270E0C6E02C10BF0F1EC0BF043
:10505000280E0C6E03C10BF0F1EC0BF000C157F5FC
:1050600001C158F502C159F503C15AF500C15BF5FC
:1050700001C15CF502C15DF503C15EF5B5EF28F035
:1050800004014D0E826F70EC0FF0290E0C6E00C102
:105090000BF0F1EC0BF000C15FF500C160F5B5EF6E
:1050A00028F004014C0E826F70EC0FF00401540ED6
:1050B000826F70EC0FF004012C0E826F70EC0FF019
:1050C00084C32AF185C32BF186C32CF187C32DF14C
:1050D00088C32EF189C32FF18AC330F18BC331F11C
:1050E0008DC332F18EC333F1010155EC3CF0CCECB1
:1050F0003BF00101000E046F000E056F010E066FFC
:10510000000E076F03EC3BF0210E0C6E00C10BF09C
:10511000F1EC0BF0220E0C6E01C10BF0F1EC0BF078
:10512000230E0C6E02C10BF0F1EC0BF0240E0C6E92
:1051300003C10BF0F1EC0BF000C161F501C162F5A8
:1051400002C163F503C164F5B5EF28F004014C0E0C
:10515000826F70EC0FF00401490E826F70EC0FF05B
:1051600004012C0E826F70EC0FF0250E08EC0CF091
:10517000E8CF00F1260E08EC0CF0E8CF01F1270E85
:1051800008EC0CF0E8CF02F1280E08EC0CF0E8CFA8
:1051900003F190EC3BF053EC39F00401730E826F95
:1051A00070EC0FF004012C0E826F70EC0FF007EC26
:1051B0003CF0290E08EC0CF0E8CF00F190EC3BF04D
:1051C00053EC39F004016D0E826F70EC0FF00401A6
:1051D0002C0E826F70EC0FF05BC500F15CC501F125
:1051E0005DC502F15EC503F190EC3BF053EC39F084
:1051F0000401730E826F70EC0FF004012C0E826FAD
:1052000070EC0FF007EC3CF060C500F190EC3BF067
:1052100053EC39F004016D0E826F70EC0FF0040155
:105220002C0E826F70EC0FF061C500F162C501F1C8
:1052300063C502F164C503F138EC34F004012C0EAF
:10524000826F70EC0FF07AEC0FF01DEF34F083C337
:105250002AF184C32BF185C32CF186C32DF187C3BA
:105260002EF188C32FF189C330F18AC331F18BC38A
:1052700032F18CC333F1010155EC3CF0CCEC3BF046
:10528000160E0C6E00C10BF0F1EC0BF0170E0C6E4D
:1052900001C10BF0F1EC0BF0180E0C6E02C10BF01B
:1052A000F1EC0BF0190E0C6E03C10BF0F1EC0BF0EE
:1052B00000C18EF101C18FF102C190F103C191F1E2
:1052C00000C192F101C193F102C194F103C195F1C2
:1052D00009EF2AF083C32AF184C32BF185C32CF193
:1052E00086C32DF187C32EF188C32FF189C330F116
:1052F0008AC331F18BC332F18CC333F1010155EC18
:105300003CF0CCEC3BF000C18EF101C18FF102C149
:1053100090F103C191F100C192F101C193F102C179
:1053200094F103C195F109EF2AF083C32AF184C3F4
:105330002BF185C32CF186C32DF187C32EF188C3D1
:105340002FF189C330F18AC331F18CC332F18DC39F
:1053500033F1010155EC3CF0CCEC3BF00101000EC7
:10536000046F000E056F010E066F000E076F03EC51
:105370003BF01A0E0C6E00C10BF0F1EC0BF01B0EA3
:105380000C6E01C10BF0F1EC0BF01C0E0C6E02C1A7
:105390000BF0F1EC0BF01D0E0C6E03C10BF0F1ECF9
:1053A0000BF000C196F101C197F102C198F103C160
:1053B00099F109EF2AF083C32AF184C32BF185C345
:1053C0002CF186C32DF187C32EF188C32FF189C339
:1053D00030F18AC331F18CC332F18DC333F1010155
:1053E00055EC3CF0CCEC3BF00101000E046F000EDC
:1053F000056F010E066F000E076F03EC3BF000C156
:1054000096F101C197F102C198F103C199F109EF39
:105410002AF0160E08EC0CF0E8CF00F1170E08EC9D
:105420000CF0E8CF01F1180E08EC0CF0E8CF02F117
:10543000190E08EC0CF0E8CF03F190EC3BF053ECC4
:1054400039F00401730E826F70EC0FF004012C0E22
:10545000826F70EC0FF08EC100F18FC101F190C12D
:1054600002F191C103F190EC3BF053EC39F00401EF
:10547000730E826F70EC0FF004012C0E826F70ECD3
:105480000FF01A0E08EC0CF0E8CF00F11B0E08EC40
:105490000CF0E8CF01F11C0E08EC0CF0E8CF02F1A3
:1054A0001D0E08EC0CF0E8CF03F138EC34F00401E9
:1054B0002C0E826F70EC0FF096C100F197C101F1D4
:1054C00098C102F199C103F138EC34F07AEC0FF095
:1054D0001DEF34F00401690E826F70EC0FF00401CF
:1054E0002C0E826F70EC0FF00101040E006F000EA5
:1054F000016F000E026F000E036F90EC3BF02CC1A9
:1055000082F40401300E822770EC0FF02DC182F47A
:105510000401300E822770EC0FF02EC182F40401DA
:10552000300E822770EC0FF02FC182F40401300E90
:10553000822770EC0FF030C182F40401300E822714
:1055400070EC0FF031C182F40401300E822770EC50
:105550000FF032C182F40401300E822770EC0FF09C
:1055600033C182F40401300E822770EC0FF0040185
:105570002C0E826F70EC0FF001010B0E006F000E0D
:10558000016F000E026F000E036F90EC3BF02CC118
:1055900082F40401300E822770EC0FF02DC182F4EA
:1055A0000401300E822770EC0FF02EC182F404014A
:1055B000300E822770EC0FF02FC182F40401300E00
:1055C000822770EC0FF030C182F40401300E822784
:1055D00070EC0FF031C182F40401300E822770ECC0
:1055E0000FF032C182F40401300E822770EC0FF00C
:1055F00033C182F40401300E822770EC0FF00401F5
:105600002C0E826F70EC0FF001014F0E006F000E38
:10561000016F000E026F000E036F90EC3BF02CC187
:1056200082F40401300E822770EC0FF02DC182F459
:105630000401300E822770EC0FF02EC182F40401B9
:10564000300E822770EC0FF02FC182F40401300E6F
:10565000822770EC0FF030C182F40401300E8227F3
:1056600070EC0FF031C182F40401300E822770EC2F
:105670000FF032C182F40401300E822770EC0FF07B
:1056800033C182F40401300E822770EC0FF0040164
:105690002C0E826F70EC0FF0200EF86EF76AF66A2F
:1056A00004010900F5CF82F470EC0FF00900F5CF8A
:1056B00082F470EC0FF00900F5CF82F470EC0FF07B
:1056C0000900F5CF82F470EC0FF00900F5CF82F4F9
:1056D00070EC0FF00900F5CF82F470EC0FF00900C8
:1056E000F5CF82F470EC0FF00900F5CF82F470EC86
:1056F0000FF07AEC0FF01DEF34F08351630AD8A459
:105700001BEF34F08451610AD8A41BEF34F08551AB
:105710006C0AD8A41BEF34F08651410A3FE0865151
:10572000440A1BE08651420AD8B4E1EF2BF08651BF
:10573000350AD8B4A7EF35F08651360AD8B4FCEF55
:1057400035F08651370AD8B465EF36F08651380AFD
:10575000D8B4C3EF36F01BEF34F00798079A040172
:105760007A0E826F70EC0FF00401780E826F70EC8D
:105770000FF00401640E826F70EC0FF00401550EFF
:10578000826F70EC0FF0CAEF2BF004014C0E826FA9
:1057900070EC0FF07AEC0FF01DEF34F00788079AE9
:1057A00004017A0E826F70EC0FF00401410E826FDB
:1057B00070EC0FF00401610E826F70EC0FF0BEEF21
:1057C0002BF00798078A04017A0E826F70EC0FF0B5
:1057D0000401420E826F70EC0FF00401610E826FC3
:1057E00070EC0FF0BEEF2BF001016667FFEF2BF0BE
:1057F0006767FFEF2BF06867FFEF2BF0696716D044
:1058000001014F670BEF2CF050670BEF2CF0516745
:105810000BEF2CF052670AD00101000E006F000E52
:10582000016F000E026F000E036F120011B80AD054
:105830000101620E046F010E056F000E066F000E6F
:10584000076F09D00101A70E046F020E056F000E4D
:10585000066F000E076F66C100F167C101F168C1F4
:1058600002F169C103F1F2EC3AF003BFA8EF2CF0AA
:10587000119A119C0101000E046FA80E056F550EC0
:10588000066F020E076F66C100F167C101F168C1C2
:1058900002F169C103F166C18AF167C18BF168C188
:1058A0008CF169C18DF1F2EC3AF003BF0BD001012C
:1058B000000E8A6FA80E8B6F550E8C6F020E8D6FC7
:1058C000118A119C0E0E08EC0CF0E8CF18F10F0EA7
:1058D00008EC0CF0E8CF19F1100E08EC0CF0E8CF52
:1058E0001AF1110E08EC0CF0E8CF1BF13BEC3AF08A
:1058F0008AC104F18BC105F18CC106F18DC107F19C
:10590000F2EC3AF00782FFEC39F03BEC3AF0079208
:10591000FFEC39F08AC100F18BC101F18CC102F1B9
:105920008DC103F10792FFEC39F0CC0E046FE00E4D
:10593000056F870E066F050E076FF2EC3AF000C197
:1059400018F101C119F102C11AF103C11BF140D0D4
:1059500013AAADEF2CF0138E139A119C119A01012A
:10596000800E006F1A0E016F060E026F000E036F9D
:105970004FC104F150C105F151C106F152C107F107
:10598000F2EC3AF003AF05D007EC3CF0118C119A21
:1059900012000E0E08EC0CF0E8CF18F10F0E08EC18
:1059A0000CF0E8CF19F1100E08EC0CF0E8CF1AF16A
:1059B000110E08EC0CF0E8CF1BF14FC100F150C103
:1059C00001F151C102F152C103F10782FFEC39F03C
:1059D00018C100F119C101F11AC102F11BC103F193
:1059E00012000784BAC166F1BBC167F1BCC168F19E
:1059F000BDC169F14BC14FF14CC150F14DC151F1E5
:105A00004EC152F157C159F158C15AF107940101E1
:105A1000666712EF2DF0676712EF2DF0686712EFDF
:105A20002DF0696716D001014F671EEF2DF050670A
:105A30001EEF2DF051671EEF2DF052670AD00101C5
:105A4000000E006F000E016F000E026F000E036F5C
:105A5000120011B80AD00101620E046F010E056F29
:105A6000000E066F000E076F09D00101A70E046F2C
:105A7000020E056F000E066F000E076F66C100F183
:105A800067C101F168C102F169C103F1F2EC3AF0BA
:105A900003BFAAEF2DF00101000E046FA80E056FE1
:105AA000550E066F020E076F66C100F167C101F166
:105AB00068C102F169C103F166C18AF167C18BF166
:105AC00068C18CF169C18DF1F2EC3AF003BF09D0E5
:105AD0000101000E8A6FA80E8B6F550E8C6F020E9F
:105AE0008D6F3BEC3AF000C104F101C105F102C138
:105AF00006F103C107F1000E006FA00E016F980EB2
:105B0000026F7B0E036F23EC3BF000C118F101C163
:105B100019F102C11AF103C11BF1000E006FA00EB2
:105B2000016F980E026F7B0E036F8AC104F18BC167
:105B300005F18CC106F18DC107F123EC3BF018C1D2
:105B400004F119C105F11AC106F11BC107F1F2EC0C
:105B50003AF012000101A80E006F610E016F000EF5
:105B6000026F000E036F4FC104F150C105F151C126
:105B700006F152C107F1F2EC3AF003AF0AD001018D
:105B8000A80E006F610E016F000E026F000E036F12
:105B900000D0C80E006FAF0E016F000E026F000E36
:105BA000036F4FC104F150C105F151C106F152C15B
:105BB00007F103EC3BF012000784BAC166F1BBC1E8
:105BC00067F1BCC168F1BDC169F14BC14FF14CC176
:105BD00050F14DC151F14EC152F157C159F158C167
:105BE0005AF1079401016667FDEF2DF06767FDEF3D
:105BF0002DF06867FDEF2DF0696716D001014F6742
:105C000009EF2EF0506709EF2EF0516709EF2EF0E3
:105C100052670AD00101000E006F000E016F000EE6
:105C2000026F000E036F120011B80AD00101620E5C
:105C3000046F010E056F000E066F000E076F09D08E
:105C40000101A70E046F020E056F000E066F000E15
:105C5000076F66C100F167C101F168C102F169C156
:105C600003F1F2EC3AF003BFBFEF2EF00101000E9A
:105C7000046FA80E056F550E066F020E076F66C102
:105C800000F167C101F168C102F169C103F166C1A8
:105C90008AF167C18BF168C18CF169C18DF1F2ECB9
:105CA0003AF003BF09D00101000E8A6FA80E8B6F76
:105CB000550E8C6F020E8D6F010E006F000E016F7E
:105CC000000E026F000E036F8AC104F18BC105F153
:105CD0008CC106F18DC107F123EC3BF018C104F132
:105CE00019C105F11AC106F11BC107F190EC3BF097
:105CF0002AC182F40401300E822770EC0FF02BC110
:105D000082F40401300E822770EC0FF02CC182F473
:105D10000401300E822770EC0FF02DC182F40401D3
:105D2000300E822770EC0FF02EC182F40401300E89
:105D3000822770EC0FF02FC182F40401300E82270D
:105D400070EC0FF030C182F40401300E822770EC49
:105D50000FF031C182F40401300E822770EC0FF095
:105D600032C182F40401300E822770EC0FF033C18F
:105D700082F40401300E822770EC0FF012004FC144
:105D800000F150C101F151C102F152C103F1010111
:105D900090EC3BF053EC39F012000401730E826F6B
:105DA00070EC0FF004012C0E826F70EC0FF0078482
:105DB00062C166F163C167F164C168F165C169F1EF
:105DC0004BC14FF14CC150F14DC151F14EC152F197
:105DD00057C159F158C15AF10794F3EC2EF07AECFF
:105DE0000FF01DEF34F066C100F167C101F168C129
:105DF00002F169C103F1010190EC3BF053EC39F081
:105E00000401630E826F70EC0FF004012C0E826FA0
:105E100070EC0FF04FC100F150C101F151C102F11E
:105E200052C103F1010190EC3BF053EC39F0040155
:105E3000660E826F70EC0FF004012C0E826F70EC16
:105E40000FF007EC3CF059C100F15AC101F101011A
:105E500090EC3BF053EC39F00401740E826F70EC5F
:105E60000FF0120010820401530E826F70EC0FF0DD
:105E700004012C0E826F70EC0FF083C32AF184C3EF
:105E80002BF185C32CF186C32DF187C32EF188C376
:105E90002FF189C330F18AC331F18BC332F18CC346
:105EA00033F1010155EC3CF0CCEC3BF000C166F164
:105EB00001C167F102C168F103C169F18EC32AF122
:105EC0008FC32BF190C32CF191C32DF192C32EF10E
:105ED00093C32FF194C330F195C331F196C332F1DE
:105EE00097C333F1010155EC3CF0CCEC3BF000C121
:105EF0004FF101C150F102C151F103C152F148EC1F
:105F00003CF099C32FF19AC330F19BC331F19CC38C
:105F100032F19DC333F1010155EC3CF0CCEC3BF088
:105F200000C159F101C15AF1F3EC2EF004012C0E1D
:105F3000826F70EC0FF0ADEF2FF0118E1CA002D02D
:105F40001CAE108C1BBE02D01BA4108E030182510C
:105F5000520A02E10F8201D00F928251750A02E1CA
:105F6000108401D010948251550A02E1108601D0AC
:105F700010968351310A03E11382138402D01392E5
:105F8000139403018351660A01E056D00401660EA2
:105F9000826F70EC0FF004012C0E826F70EC0FF02A
:105FA000F1EC2CF090EC3BF02AC182F40401300EAD
:105FB000822770EC0FF02BC182F40401300E82278F
:105FC00070EC0FF02CC182F40401300E822770ECCB
:105FD0000FF02DC182F40401300E822770EC0FF017
:105FE0002EC182F40401300E822770EC0FF02FC115
:105FF00082F40401300E822770EC0FF030C182F47D
:106000000401300E822770EC0FF031C182F40401DC
:10601000300E822770EC0FF032C182F40401300E92
:10602000822770EC0FF033C182F40401300E822716
:1060300070EC0FF01BEF34F011A003D011A401D0CD
:106040001084078410B286EF30F010A46AEF30F0AD
:10605000BAC166F1BBC167F1BCC168F1BDC169F1EC
:10606000BEC16AF1BFC16BF1C0C16CF1C1C16DF1BC
:10607000C2C16EF1C3C16FF1C4C170F1C5C171F18C
:10608000C6C172F1C7C173F1C8C174F1C9C175F15C
:10609000CAC176F1CBC177F1CCC178F1CDC179F12C
:1060A000CEC17AF1CFC17BF1D0C17CF1D1C17DF1FC
:1060B000D2C17EF1D3C17FF1D4C180F1D5C181F1CC
:1060C000D6C182F1D7C183F1D8C184F1D9C185F19C
:1060D00072EF30F062C166F163C167F164C168F1CB
:1060E00065C169F1BAC186F1BBC187F1BCC188F154
:1060F000BDC189F14BC14FF14CC150F14DC151F1BE
:106100004EC152F157C159F158C15AF107940FA02D
:10611000A8EF30F00101966795EF30F0976795EFA3
:1061200030F0986795EF30F0996799EF30F0A8EF6D
:1061300030F0F4EC2BF096C104F197C105F198C151
:1061400006F199C107F1F2EC3AF003BFE1EF33F049
:10615000F4EC2BF00101000E046F000E056F010E30
:10616000066F000E076F23EC3BF011A02AD011A29E
:1061700028D090EC3BF0296701D005D004012D0E0A
:10618000826F70EC0FF030C182F40401300E822770
:1061900070EC0FF031C182F40401300E822770ECF4
:1061A0000FF032C182F40401300E822770EC0FF040
:1061B00033C182F40401300E822770EC0FF07AECC8
:1061C0000FF012A8C5D012981DC01EF01E3A1E4234
:1061D000070E1E1600011E50000AD8B474EF31F0ED
:1061E00000011E50010AD8B400EF31F000011E502A
:1061F000020AD8B4FEEF30F0A6EF31F0A6EF31F08E
:1062000007EC3CF02DC001F12EC000F1D890013315
:106210000033D890013300330101630E046F000E88
:10622000056F000E066F000E076F23EC3BF0280E83
:10623000046F000E056F000E066F000E076FF2EC84
:106240003AF000C130F007EC3CF02BC001F1019FA7
:10625000019D2CC000F10101A40E046F000E056F1A
:10626000000E066F000E076F23EC3BF000C12FF00D
:1062700000C104F101C105F102C106F103C107F13A
:10628000640E006F000E016F000E026F000E036FB0
:10629000F2EC3AF0050E046F000E056F000E066F6B
:1062A000000E076F23EC3BF000C104F101C105F1C2
:1062B00002C106F103C107F107EC3CF030C000F168
:1062C000F2EC3AF000C131F031C0E8FF050F305C6C
:1062D00003E78A84A6EF31F031C0E8FF0A0F305C93
:1062E00001E68A94A6EF31F000C124F101C125F145
:1062F00002C126F103C127F107EC3CF00DEC3CF0A4
:106300001D501F0BE8CF00F10101640E046F000E59
:10631000056F000E066F000E076F03EC3BF024C103
:1063200004F125C105F126C106F127C107F1F2EC00
:106330003AF003BF02D08A9401D08A8424C100F1CC
:1063400025C101F126C102F127C103F11DEF34F08F
:1063500000C124F101C125F102C126F103C127F1D9
:1063600010AE4DD0109E00C108F101C109F102C16B
:106370000AF103C10BF190EC3BF030C1E2F131C105
:10638000E3F132C1E4F133C1E5F108C100F109C123
:1063900001F10AC102F10BC103F101016C0E046F9E
:1063A000070E056F000E066F000E076FF2EC3AF055
:1063B00003BF04D00101550EE66F1CD008C100F1E7
:1063C00009C101F10AC102F10BC103F10101A40EDF
:1063D000046F060E056F000E066F000E076FF2ECDD
:1063E0003AF003BF04D001017F0EE66F03D0010134
:1063F000FF0EE66F1F8E11AEE1EF33F0119E24C148
:1064000000F125C101F126C102F127C103F111A05C
:1064100005D011A203D00FB0E1EF33F010A418EFB4
:1064200032F00401750E826F70EC0FF01DEF32F048
:106430000401720E826F70EC0FF004012C0E826F5B
:1064400070EC0FF090EC3BF029672CEF32F0040178
:10645000200E826F2FEF32F004012D0E826F70EC50
:106460000FF030C182F40401300E822770EC0FF07F
:1064700031C182F40401300E822770EC0FF0040168
:106480002E0E826F70EC0FF032C182F40401300ED8
:10649000822770EC0FF033C182F40401300E8227A2
:1064A00070EC0FF004016D0E826F70EC0FF00401C0
:1064B0002C0E826F70EC0FF04FC100F150C101F152
:1064C00051C102F152C103F1010190EC3BF053ECD8
:1064D00039F00401480E826F70EC0FF004017A0E5F
:1064E000826F70EC0FF004012C0E826F70EC0FF0D5
:1064F00066C100F167C101F168C102F169C103F130
:10650000010190EC3BF053EC39F00401630E826F13
:1065100070EC0FF004012C0E826F70EC0FF066C16E
:1065200000F167C101F168C102F169C103F1010124
:106530000A0E046F000E056F000E066F000E076F47
:1065400003EC3BF0000E046F120E056F000E066F99
:10655000000E076F23EC3BF090EC3BF02AC182F475
:106560000401300E822770EC0FF02BC182F404017D
:10657000300E822770EC0FF02CC182F40401300E33
:10658000822770EC0FF02DC182F40401300E8227B7
:1065900070EC0FF02EC182F40401300E822770ECF3
:1065A0000FF02FC182F40401300E822770EC0FF03F
:1065B00030C182F40401300E822770EC0FF0040128
:1065C0002E0E826F70EC0FF031C182F40401300E98
:1065D000822770EC0FF032C182F40401300E822762
:1065E00070EC0FF033C182F40401300E822770EC9E
:1065F0000FF00401730E826F70EC0FF004012C0E8B
:10660000826F70EC0FF007EC3CF059C100F15AC1F9
:1066100001F147EC35F013A25DEF33F004012C0ECD
:10662000826F70EC0FF086C166F187C167F188C197
:1066300068F189C169F1F4EC2BF00101000E046FDF
:10664000000E056F010E066F000E076F23EC3BF086
:1066500090EC3BF0296732EF33F00401200E826F9B
:1066600035EF33F004012D0E826F70EC0FF030C166
:1066700082F40401300E822770EC0FF031C182F4F5
:106680000401300E822770EC0FF004012E0E826F91
:1066900070EC0FF032C182F40401300E822770ECEE
:1066A0000FF033C182F40401300E822770EC0FF03A
:1066B00004016D0E826F70EC0FF003018351460AE6
:1066C00001E007D004012C0E826F70EC0FF0DCECBF
:1066D0002DF013A490EF33F004012C0E826F70ECB8
:1066E0000FF013AC7EEF33F00401500E826F70ECAC
:1066F0000FF0139C1398139A90EF33F013AE8BEFB7
:1067000033F00401460E826F70EC0FF0139E139865
:10671000139A90EF33F00401530E826F70EC0FF078
:1067200037B0A7EF33F004012C0E826F70EC0FF03E
:106730008BB0A2EF33F00401440E826F70EC0FF0C7
:10674000A7EF33F00401530E826F70EC0FF00FB21D
:10675000ADEF33F00FA0DFEF33F004012C0E826FAA
:1067600070EC0FF0200EF86EF76AF66A040109006B
:10677000F5CF82F470EC0FF00900F5CF82F470ECE5
:106780000FF00900F5CF82F470EC0FF00900F5CF9F
:1067900082F470EC0FF00900F5CF82F470EC0FF08A
:1067A0000900F5CF82F470EC0FF00900F5CF82F408
:1067B00070EC0FF00900F5CF82F470EC0FF07AEC7A
:1067C0000FF00F90109E12981DEF34F00401630E2D
:1067D000826F70EC0FF004012C0E826F70EC0FF0E2
:1067E00023EC34F004012C0E826F70EC0FF096EC69
:1067F00034F004012C0E826F70EC0FF012EC35F0C7
:1068000004012C0E826F70EC0FF00101F80E006F86
:10681000CD0E016F660E026F030E036F38EC34F07D
:1068200004012C0E826F70EC0FF028EC35F07AEC3E
:106830000FF01DEF34F07AEC0FF00301C26B0790FC
:1068400010922CEF37F0D8900E0E08EC0CF0E8CF39
:1068500000F10F0E08EC0CF0E8CF01F1100E08EC7F
:106860000CF0E8CF02F1110E08EC0CF0E8CF03F1C8
:106870000101000E046F000E056F010E066F000E81
:10688000076F23EC3BF090EC3BF02AC182F404014B
:10689000300E822770EC0FF02BC182F40401300E11
:1068A000822770EC0FF02CC182F40401300E822795
:1068B00070EC0FF02DC182F40401300E822770ECD1
:1068C0000FF02EC182F40401300E822770EC0FF01D
:1068D0002FC182F40401300E822770EC0FF030C11A
:1068E00082F40401300E822770EC0FF031C182F483
:1068F0000401300E822770EC0FF004012E0E826F1F
:1069000070EC0FF032C182F40401300E822770EC7B
:106910000FF033C182F40401300E822770EC0FF0C7
:1069200004016D0E826F70EC0FF01200120E08EC75
:106930000CF0E8CF00F1130E08EC0CF0E8CF01F1F9
:10694000140E08EC0CF0E8CF02F1150E08EC0CF078
:10695000E8CF03F101010A0E046F000E056F000E6F
:10696000066F000E076F03EC3BF0000E046F120E73
:10697000056F000E066F000E076F23EC3BF090ECE6
:106980003BF02AC182F40401300E822770EC0FF034
:106990002BC182F40401300E822770EC0FF02CC161
:1069A00082F40401300E822770EC0FF02DC182F4C6
:1069B0000401300E822770EC0FF02EC182F4040126
:1069C000300E822770EC0FF02FC182F40401300EDC
:1069D000822770EC0FF030C182F40401300E822760
:1069E00070EC0FF004012E0E826F70EC0FF031C1CD
:1069F00082F40401300E822770EC0FF032C182F471
:106A00000401300E822770EC0FF033C182F40401D0
:106A1000300E822770EC0FF00401730E826F70EC61
:106A20000FF012000A0E08EC0CF0E8CF00F10B0E8C
:106A300008EC0CF0E8CF01F10C0E08EC0CF0E8CFFC
:106A400002F10D0E08EC0CF0E8CF03F147EF35F042
:106A5000060E08EC0CF0E8CF00F1070E08EC0CF085
:106A6000E8CF01F1080E08EC0CF0E8CF02F1090EB6
:106A700008EC0CF0E8CF03F147EF35F0010107EC2B
:106A80003CF0078457C100F158C101F1079401019E
:106A9000E80E046F800E056F000E066F000E076F84
:106AA00003EC3BF0000E046F040E056F000E066F42
:106AB000000E076F23EC3BF0880E046F130E056F7A
:106AC000000E066F000E076FF2EC3AF00A0E046F2C
:106AD000000E056F000E066F000E076F23EC3BF0F3
:106AE00090EC3BF0010129677BEF35F00401200EAB
:106AF000826F7EEF35F004012D0E826F70EC0FF087
:106B000030C182F40401300E822770EC0FF031C1E5
:106B100082F40401300E822770EC0FF032C182F44F
:106B20000401300E822770EC0FF004012E0E826FEC
:106B300070EC0FF033C182F40401300E822770EC48
:106B40000FF00401430E826F70EC0FF0120087C348
:106B50002AF188C32BF189C32CF18AC32DF18BC391
:106B60002EF18CC32FF18DC330F18EC331F190C360
:106B700032F191C333F10101296B55EC3CF0CCECBF
:106B80003BF00101000E046F000E056F010E066F51
:106B9000000E076F03EC3BF00E0E0C6E00C10BF005
:106BA000F1EC0BF00F0E0C6E01C10BF0F1EC0BF0E1
:106BB000100E0C6E02C10BF0F1EC0BF0110E0C6E0E
:106BC00003C10BF0F1EC0BF004017A0E826F70EC54
:106BD0000FF004012C0E826F70EC0FF00401350EE3
:106BE000826F70EC0FF004012C0E826F70EC0FF0CE
:106BF00023EC34F0CAEF2BF087C32AF188C32BF1C2
:106C000089C32CF18AC32DF18BC32EF18CC32FF1D4
:106C10008DC330F18EC331F190C332F191C333F1A2
:106C20000101296B55EC3CF0CCEC3BF0880E046F75
:106C3000130E056F000E066F000E076FF7EC3AF0AB
:106C4000000E046F040E056F000E066F000E076F36
:106C500003EC3BF00101E80E046F800E056F000E9F
:106C6000066F000E076F23EC3BF00A0E0C6E00C19E
:106C70000BF0F1EC0BF00B0E0C6E01C10BF0F1EC14
:106C80000BF00C0E0C6E02C10BF0F1EC0BF00D0EC4
:106C90000C6E03C10BF0F1EC0BF004017A0E826F65
:106CA00070EC0FF004012C0E826F70EC0FF00401F9
:106CB000360E826F70EC0FF004012C0E826F70ECB8
:106CC0000FF012EC35F0CAEF2BF087C32AF188C31E
:106CD0002BF189C32CF18AC32DF18BC32EF18CC308
:106CE0002FF18DC330F18FC331F190C332F191C3D5
:106CF00033F1010155EC3CF0CCEC3BF0000E046F9D
:106D0000120E056F000E066F000E076F03EC3BF0CE
:106D100001010A0E046F000E056F000E066F000ED3
:106D2000076F23EC3BF0120E0C6E00C10BF0F1EC80
:106D30000BF0130E0C6E01C10BF0F1EC0BF0140E06
:106D40000C6E02C10BF0F1EC0BF0150E0C6E03C1D2
:106D50000BF0F1EC0BF004017A0E826F70EC0FF087
:106D600004012C0E826F70EC0FF00401370E826F5D
:106D700070EC0FF004012C0E826F70EC0FF096ECAB
:106D800034F0CAEF2BF087C32AF188C32BF189C3F3
:106D90002CF18AC32DF18BC32EF18CC32FF18DC33F
:106DA00030F18EC331F190C332F191C333F101015F
:106DB000296B55EC3CF0CCEC3BF0880E046F130EC5
:106DC000056F000E066F000E076FF7EC3AF0000E2D
:106DD000046F040E056F000E066F000E076F03ECC4
:106DE0003BF00101E80E046F800E056F000E066F88
:106DF000000E076F23EC3BF0060E0C6E00C10BF08B
:106E0000F1EC0BF0070E0C6E01C10BF0F1EC0BF086
:106E1000080E0C6E02C10BF0F1EC0BF0090E0C6EBB
:106E200003C10BF0F1EC0BF004017A0E826F70ECF1
:106E30000FF004012C0E826F70EC0FF00401380E7D
:106E4000826F70EC0FF004012C0E826F70EC0FF06B
:106E500028EC35F0CAEF2BF007A89FEF37F00101BF
:106E6000800E006F1A0E016F060E026F000E036F88
:106E70004BC104F14CC105F14DC106F14EC107F102
:106E8000F2EC3AF003BFE5EF37F04DEC39F04BC1CF
:106E900000F14CC101F14DC102F14EC103F1078275
:106EA000FFEC39F018C104F119C105F11AC106F15E
:106EB0001BC107F1F80E006FCD0E016F660E026F59
:106EC000030E036FF2EC3AF00E0E0C6E00C10BF0E5
:106ED000F1EC0BF00F0E0C6E01C10BF0F1EC0BF0AE
:106EE000100E0C6E02C10BF0F1EC0BF0110E0C6EDB
:106EF00003C10BF0F1EC0BF00784010107EC3CF04F
:106F000057C100F158C101F107940A0E0C6E00C17F
:106F10000BF0F1EC0BF00B0E0C6E01C10BF0F1EC71
:106F20000BF00C0E0C6E02C10BF0F1EC0BF00D0E21
:106F30000C6E03C10BF0F1EC0BF0E5EF37F007AA94
:106F4000E5EF37F00784010107EC3CF057C100F191
:106F500058C101F10794060E0C6E00C10BF0F1EC64
:106F60000BF0070E0C6E01C10BF0F1EC0BF0080EEC
:106F70000C6E02C10BF0F1EC0BF0090E0C6E03C1AC
:106F80000BF0F1EC0BF0078462C100F163C101F179
:106F900064C102F165C103F10794120E0C6E00C1C9
:106FA0000BF0F1EC0BF0130E0C6E01C10BF0F1ECD9
:106FB0000BF0140E0C6E02C10BF0F1EC0BF0150E81
:106FC0000C6E03C10BF0F1EC0BF00798079A04016B
:106FD000805181197F0B0DE09EA8FED714EE00F0C2
:106FE00081517F0BE126E750812B0F01AD6EE7EF5A
:106FF00037F005012F51000AD8B428EF38F081BAD4
:107000000DEF38F015B228EF38F005012F51010AC5
:10701000D8B426EF38F01FEF38F005012F51000AE1
:10702000D8B400EF47F005012F51010AD8B426EF7C
:1070300038F000011650050AD8B400EF47F081B8C7
:1070400028EF38F088EC3EF086EC3FF099EC46F003
:1070500099EF0EF006013251385D3351D8A0010F7F
:10706000395D800BD8A439EF38F032C638F633C614
:1070700039F6120006013251365D3351D8A0010FA6
:10708000375D800BD8B449EF38F032C636F633C6D8
:1070900037F6120007841AC632F61BC633F61CC632
:1070A00038F61DC639F62AEC38F01EC632F61FC671
:1070B00033F62AEC38F020C632F621C633F62AEC35
:1070C00038F01AC632F61BC633F61CC636F61DC695
:1070D00037F63AEC38F01EC632F61FC633F63AECF5
:1070E00038F020C632F621C633F63AEC38F0385183
:1070F000365F3951D8A03929375F07EC3CF036C6E6
:1071000000F137C601F113EC3CF000C13AF601C1C1
:107110003BF622C632F623C633F624C638F625C619
:1071200039F62AEC38F026C632F627C633F62AECB2
:1071300038F028C632F629C633F62AEC38F022C6D3
:1071400032F623C633F624C636F625C637F63AECB1
:1071500038F026C632F627C633F63AEC38F028C6A1
:1071600032F629C633F63AEC38F03851365F3951E9
:10717000D8A03929375F07EC3CF036C600F137C696
:1071800001F113EC3CF000C13CF601C13DF62AC60A
:1071900032F62BC633F62CC638F62DC639F62AEC55
:1071A00038F02EC632F62FC633F62AEC38F030C649
:1071B00032F631C633F62AEC38F02AC632F62BC640
:1071C00033F62CC636F62DC637F63AEC38F02EC616
:1071D00032F62FC633F63AEC38F030C632F631C606
:1071E00033F63AEC38F03851365F3951D8A03929A6
:1071F000375F07EC3CF036C600F137C601F113ECFF
:107200003CF000C13EF601C13FF63AC632F63BC63D
:1072100033F63CC636F63DC637F63AEC38F03EC695
:1072200032F63FC633F63AEC38F00794120018C134
:1072300000F119C101F11AC102F11BC103F1000EE5
:10724000046F000E056F010E066F000E076F23EC32
:107250003BF029A142EF39F02051D8B442EF39F088
:1072600018C100F119C101F11AC102F11BC103F1EA
:10727000000E046F000E056F0A0E066F000E076FFA
:1072800023EC3BF0120001010451001305510113DE
:10729000065102130751031312000101186B196BF9
:1072A0001A6B1B6B12002AC182F40401300E822774
:1072B00070EC0FF02BC182F40401300E822770ECC9
:1072C0000FF02CC182F40401300E822770EC0FF015
:1072D0002DC182F40401300E822770EC0FF02EC114
:1072E00082F40401300E822770EC0FF02FC182F47B
:1072F0000401300E822770EC0FF030C182F40401DB
:10730000300E822770EC0FF031C182F40401300E90
:10731000822770EC0FF032C182F40401300E822714
:1073200070EC0FF033C182F40401300E822770EC50
:107330000FF012002FC182F40401300E822770EC8E
:107340000FF030C182F40401300E822770EC0FF090
:1073500031C182F40401300E822770EC0FF032C18B
:1073600082F40401300E822770EC0FF033C182F4F6
:107370000401300E822770EC0FF01200060E216E11
:10738000060E226E060E236E212EC4EF39F0222E39
:10739000C4EF39F0232EC4EF39F08B84020E216E36
:1073A000020E226E020E236E212ED4EF39F0222E11
:1073B000D4EF39F0232ED4EF39F08B941200FF0E66
:1073C000226E22C023F0030E216E8B84212EE5EF66
:1073D00039F0030E216E232EE5EF39F08B9422C095
:1073E00023F0030E216E212EF3EF39F0030E216EF0
:1073F000233EF3EF39F0222EE1EF39F012000101C4
:10740000005305E1015303E1025301E1002BC2ECFB
:107410003AF007EC3CF03951006F3A51016F420EDF
:10742000046F4B0E056F000E066F000E076F03EC26
:107430003BF000C104F101C105F102C106F103C135
:1074400007F118C100F119C101F11AC102F11BC104
:1074500003F107B230EF3AF0F7EC3AF032EF3AF0DE
:10746000F2EC3AF000C118F101C119F102C11AF1B0
:1074700003C11BF1120007EC3CF059C100F15AC1E5
:1074800001F1060E08EC0CF0E8CF04F1070E08EC51
:107490000CF0E8CF05F1080E08EC0CF0E8CF06F18F
:1074A000090E08EC0CF0E8CF07F1F2EC3AF000C15D
:1074B00024F101C125F102C126F103C127F1290EF2
:1074C000046F000E056F000E066F000E076F03ECD1
:1074D0003BF0EE0E046F430E056F000E066F000EBC
:1074E000076FF7EC3AF024C104F125C105F126C17C
:1074F00006F127C107F103EC3BF000C11CF101C10B
:107500001DF102C11EF103C11FF1120E08EC0CF0B7
:10751000E8CF04F1130E08EC0CF0E8CF05F1140EDF
:1075200008EC0CF0E8CF06F1150E08EC0CF0E8CFF3
:1075300007F10D0E006F000E016F000E026F000EBE
:10754000036F03EC3BF0180E046F000E056F000E86
:10755000066F000E076F23EC3BF01CC104F11DC148
:1075600005F11EC106F11FC107F1F7EC3AF06A0EF2
:10757000046F2A0E056F000E066F000E076FF2EC07
:107580003AF01200BF0EFA6E200E3A6F396BD890A7
:107590000037013702370337D8B0D3EF3AF03A2F2C
:1075A000C8EF3AF039073A070353D8B41200033151
:1075B000070B80093F6F03390F0B010F396F80EC08
:1075C0005FF0406F390580EC5FF0405D405F396BE4
:1075D0003F33D8B0392739333FA9E8EF3AF040516B
:1075E0003927120001012CEC3CF0D8B01200010147
:1075F00003510719346FEFEC3BF0D8900751031992
:1076000034AF800F12000101346B13EC3CF0D8A0B2
:1076100029EC3CF0D8B01200FEEC3BF007EC3CF05B
:107620001F0E366F3FEC3CF00B35D8B0EFEC3BF063
:10763000D8A00335D8B01200362F12EF3BF034B18A
:1076400016EC3CF012000101346B045105110611D7
:1076500007110008D8A013EC3CF0D8A029EC3CF0AE
:10766000D8B01200086B096B0A6B0B6B3FEC3CF057
:107670001F0E366F3FEC3CF007510B5DD8A44DEF69
:107680003BF006510A5DD8A44DEF3BF00551095D72
:10769000D8A44DEF3BF00451085DD8A060EF3BF05B
:1076A0000451085F0551D8A0053D095F0651D8A0D7
:1076B000063D0A5F0751D8A0073D0B5FD8900081B7
:1076C000362F3AEF3BF034B116EC3CF0346B13EC50
:1076D0003CF0D89043EC3CF007510B5DD8A47DEF13
:1076E0003BF006510A5DD8A47DEF3BF00551095DE2
:1076F000D8A47DEF3BF00451085DD8A08CEF3BF09F
:10770000003F8CEF3BF0013F8CEF3BF0023F8CEFF2
:107710003BF0032BD8B4120034B116EC3CF012004D
:107720000101346B13EC3CF0D8B0120048EC3CF093
:10773000200E366F003701370237033711EE33F072
:107740000A0E376FE7360A0EE75CD8B0E76EE552EF
:10775000372FA2EF3BF0362F9AEF3BF034B129815F
:10776000D890120048EC3CF0200E366F00370137FD
:107770000237033711EE33F00A0E376FE7360A0E81
:10778000E75CD8B0E76EE552372FBEEF3BF0362FFF
:10779000B6EF3BF0D890120001010A0E346F200EB4
:1077A000366F11EE29F03451376F0A0ED890E65239
:1077B000D8B0E726E732372FD7EF3BF00333023359
:1077C00001330033362FD1EF3BF0E750FF0FD8A045
:1077D0000335D8B0120029B116EC3CF01200045168
:1077E00000270551D8B0053D01270651D8B0063D08
:1077F00002270751D8B0073D032712000051086F38
:107800000151096F02510A6F03510B6F1200010100
:10781000006B016B026B036B12000101046B056BC3
:10782000066B076B12000335D8A012000351800BC2
:10783000001F011F021F031F003F26EF3CF0013F06
:1078400026EF3CF0023F26EF3CF0032B342B0325C0
:1078500012000735D8A012000751800B041F051F26
:10786000061F071F043F3CEF3CF0053F3CEF3CF098
:10787000063F3CEF3CF0072B342B07251200003766
:10788000013702370337083709370A370B37120039
:107890000101296B2A6B2B6B2C6B2D6B2E6B2F6BC5
:1078A000306B316B326B336B120001012A510F0BBD
:1078B0002A6F2B510F0B2B6F2C510F0B2C6F2D514F
:1078C0000F0B2D6F2E510F0B2E6F2F510F0B2F6F94
:1078D00030510F0B306F31510F0B316F32510F0B95
:1078E000326F33510F0B336F120000C124F101C10D
:1078F00025F102C126F103C127F104C100F105C140
:1079000001F106C102F107C103F124C104F125C14F
:1079100005F126C106F127C107F11200899C000E6E
:10792000C76E200EC66E9E96C69EC50EC96EFF0E11
:107930009EB602D0E82EFCD79E96C69E000EC96E5B
:10794000FF0E9EB602D0E82EFCD7C9CF00F69E9659
:10795000C69E000EC96EFF0E9EB602D0E82EFCD762
:10796000C9CF01F6898C1200000EC76E200EC66EBC
:10797000899C9E96C69EC80EC96EFF0E9EB602D00A
:10798000E82EFCD79E96C69E000EC96EFF0E9EB6D0
:1079900002D0E82EFCD7C9CF02F69E96C69E000EF6
:1079A000C96EFF0E9EB602D0E82EFCD7C9CF03F6F3
:1079B0009E96C69E000EC96EFF0E9EB602D0E82EA1
:1079C000FCD7C9CF0AF69E96C69E000EC96EFF0E62
:1079D0009EB602D0E82EFCD7C9CF0BF69E96C69E67
:1079E000000EC96EFF0E9EB602D0E82EFCD7C9CF9E
:1079F00012F69E96C69E000EC96EFF0E9EB602D06F
:107A0000E82EFCD7C9CF13F6898C1200000EC76E82
:107A1000200EC66E899C9E96C69EE80EC96EFF0E0D
:107A20009EB602D0E82EFCD79E96C69E000EC96E6A
:107A3000FF0E9EB602D0E82EFCD7C9CF1AF69E964E
:107A4000C69E000EC96EFF0E9EB602D0E82EFCD771
:107A5000C9CF1BF69E96C69E000EC96EFF0E9EB63F
:107A600002D0E82EFCD7C9CF22F69E96C69E000E05
:107A7000C96EFF0E9EB602D0E82EFCD7C9CF23F602
:107A80009E96C69E000EC96EFF0E9EB602D0E82ED0
:107A9000FCD7C9CF2AF69E96C69E000EC96EFF0E71
:107AA0009EB602D0E82EFCD7C9CF2BF6898C1200E7
:107AB000000EC76E200EC66E899C9E96C69E240E32
:107AC000C96EFF0E9EB602D0E82EFCD79E96C69ECB
:107AD000E40EC96EFF0E9EB602D0E82EFCD7898C4C
:107AE000899C9E96C69E200EC96EFF0E9EB602D041
:107AF000E82EFCD79E96C69E5F0EC96EFF0E9EB600
:107B000002D0E82EFCD7898C899C9E96C69E210EB9
:107B1000C96EFF0E9EB602D0E82EFCD79E96C69E7A
:107B2000C00EC96EFF0E9EB602D0E82EFCD7898C1F
:107B3000899C9E96C69E260EC96EFF0E9EB602D0EA
:107B4000E82EFCD79E96C69E000EC96EFF0E9EB60E
:107B500002D0E82EFCD7898C1200000EC76E200ED2
:107B6000C66E899C9E96C69E200EC96EFF0E9EB65E
:107B700002D0E82EFCD79E96C69E000EC96EFF0E60
:107B80009EB602D0E82EFCD7898C120010A806D031
:107B90008994000EC76E220EC66E05D08984000E31
:107BA000C76E220EC66E050EE82EFED7120010A874
:107BB00002D0898401D08994050EE82EFED71200E8
:107BC000C6EC3DF09E96C69E000EC96EFF0E9EB698
:107BD00002D0E82EFCD79E96C69E000EC96EFF0E00
:107BE0009EB602D0E82EFCD7C9CFAFF59E96C69EB2
:107BF000000EC96EFF0E9EB602D0E82EFCD7C9CF8C
:107C0000B0F59E96C69E000EC96EFF0E9EB602D0BF
:107C1000E82EFCD7C9CFB1F59E96C69E000EC96E60
:107C2000FF0E9EB602D0E82EFCD7C9CFB2F59E96C5
:107C3000C69E000EC96EFF0E9EB602D0E82EFCD77F
:107C4000C9CFB3F59E96C69E000EC96EFF0E9EB6B6
:107C500002D0E82EFCD7C9CFB4F59E96C69E000E82
:107C6000C96EFF0E9EB602D0E82EFCD7C9CFB5F57F
:107C7000D7EC3DF01200C6EC3DF09E96C69E800EFD
:107C8000C96EFF0E9EB602D0E82EFCD79E96C69E09
:107C9000AFC5C9FFFF0E9EB602D0E82EFCD79E9658
:107CA000C69EB0C5C9FFFF0E9EB602D0E82EFCD717
:107CB0009E96C69EB1C5C9FFFF0E9EB602D0E82EA5
:107CC000FCD79E96C69EB2C5C9FFFF0E9EB602D0D7
:107CD000E82EFCD79E96C69EB3C5C9FFFF0E9EB682
:107CE00002D0E82EFCD79E96C69EB4C5C9FFFF0EF3
:107CF0009EB602D0E82EFCD79E96C69EB5C5C9FF9B
:107D0000FF0E9EB602D0E82EFCD7D7EC3DF0120055
:107D1000C6EC3DF09E96C69E070EC96EFF0E9EB63F
:107D200002D0E82EFCD79E96C69E000EC96EFF0EAE
:107D30009EB602D0E82EFCD7C9CFAFF59E96C69E60
:107D4000000EC96EFF0E9EB602D0E82EFCD7C9CF3A
:107D5000B0F59E96C69E000EC96EFF0E9EB602D06E
:107D6000E82EFCD7C9CFB1F59E96C69E000EC96E0F
:107D7000FF0E9EB602D0E82EFCD7C9CFB2F5D7ECE5
:107D80003DF0C6EC3DF09E96C69E25C0C9FFFF0E95
:107D90009EB602D0E82EFCD79E96C69E000EC96EF7
:107DA000FF0E9EB602D0E82EFCD7C9CFB6F5D7ECB1
:107DB0003DF01200C6EC3DF09E96C69E870EC96E41
:107DC000FF0E9EB602D0E82EFCD79E96C69EAFC58B
:107DD000C9FFFF0E9EB602D0E82EFCD79E96C69E27
:107DE000B0C5C9FFFF0E9EB602D0E82EFCD79E9606
:107DF000C69EB1C5C9FFFF0E9EB602D0E82EFCD7C5
:107E00009E96C69EB2C5C9FFFF0E9EB602D0E82E52
:107E1000FCD7D7EC3DF0C6EC3DF09E96C69E26C042
:107E2000C9FFFF0E9EB602D0E82EFCD79E96C69ED6
:107E3000B6C5C9FFFF0E9EB602D0E82EFCD7D7EC20
:107E40003DF01200C6EC3DF09E96C69E870EC96EB0
:107E5000FF0E9EB602D0E82EFCD79E96C69E000E60
:107E6000C96EFF0E9EB602D0E82EFCD79E96C69E27
:107E7000800EC96EFF0E9EB602D0E82EFCD79E96ED
:107E8000C69E800EC96EFF0E9EB602D0E82EFCD7AD
:107E90009E96C69E800EC96EFF0E9EB602D0E82E3C
:107EA000FCD7D7EC3DF01200C6EC3DF09E96C69E86
:107EB000870EC96EFF0E9EB602D0E82EFCD79E96A6
:107EC000C69E000EC96EFF0E9EB602D0E82EFCD7ED
:107ED0009E96C69E000EC96EFF0E9EB602D0E82E7C
:107EE000FCD79E96C69E800EC96EFF0E9EB602D02F
:107EF000E82EFCD79E96C69E800EC96EFF0E9EB6DB
:107F000002D0E82EFCD7D7EC3DF0120010A817D015
:107F1000C6EC3DF09E96C69E8F0EC96EFF0E9EB6B5
:107F200002D0E82EFCD79E96C69E000EC96EFF0EAC
:107F30009EB602D0E82EFCD7D7EC3DF0120088ECBC
:107F40003EF0120010A82DD0C6EC3DF09E96C69EC5
:107F500026C0C9FFFF0E9EB602D0E82EFCD79E9623
:107F6000C69E450EC96EFF0E9EB602D0E82EFCD707
:107F7000D7EC3DF0C6EC3DF09E96C69E8F0EC96EC6
:107F8000FF0E9EB602D0E82EFCD79E96C69E000E2F
:107F9000C96EFF0E9EB602D0E82EFCD7D7EC3DF09E
:107FA0001200C6EC3DF09E96C69E26C0C9FFFF0E8D
:107FB0009EB602D0E82EFCD79E96C69E010EC96ED4
:107FC000FF0E9EB602D0E82EFCD7D7EC3DF0C6ECF3
:107FD0003DF09E96C69E910EC96EFF0E9EB602D0D3
:107FE000E82EFCD79E96C69EA50EC96EFF0E9EB6C5
:107FF00002D0E82EFCD7D7EC3DF01200C6EC3DF0E5
:108000009E96C69E26C0C9FFFF0E9EB602D0E82EE1
:10801000FCD79E96C69E810EC96EFF0E9EB602D0FC
:10802000E82EFCD7D7EC3DF01200C6EC3DF09E9652
:10803000C69E26C0C9FFFF0E9EB602D0E82EFCD712
:108040009E96C69E010EC96EFF0E9EB602D0E82E09
:10805000FCD7D7EC3DF01200C6EC3DF09E96C69ED4
:10806000910EC96EFF0E9EB602D0E82EFCD79E96EA
:10807000C69EA50EC96EFF0E9EB602D0E82EFCD796
:10808000D7EC3DF01200C6EC3DF09E96C69E910ED8
:10809000C96EFF0E9EB602D0E82EFCD79E96C69EF5
:1080A000000EC96EFF0E9EB602D0E82EFCD7D7ECAC
:1080B0003DF012000501256B266B276B286B899A12
:1080C000400EC76E200EC66E9E96C69E030EC96EEB
:1080D000FF0E9EB602D0E82EFCD79E96C69E27C500
:1080E000C9FFFF0E9EB602D0E82EFCD79E96C69E14
:1080F00026C5C9FFFF0E9EB602D0E82EFCD79E967D
:10810000C69E25C5C9FFFF0E9EB602D0E82EFCD73D
:108110009E96C69EC952FF0E9EB602D0E82EFCD790
:10812000898A0F01C950FF0A01E1120005012E5191
:10813000130A05E005012E51170A0CE01200050193
:10814000E00E256FFF0E266F0F0E276F000E286FB3
:10815000B3EF40F00501E00E256FFF0E266FFF0E16
:10816000276F000E286F899A400EC76E200EC66ECC
:108170009E96C69E030EC96EFF0E9EB602D0E82ED6
:10818000FCD79E96C69E27C5C9FFFF0E9EB602D09D
:10819000E82EFCD79E96C69E26C5C9FFFF0E9EB64A
:1081A00002D0E82EFCD79E96C69E25C5C9FFFF0EBD
:1081B0009EB602D0E82EFCD79E96C69EC952FF0EF0
:1081C0009EB602D0E82EFCD7898A0F01C950FF0A5B
:1081D0001DE005012E51130A05E005012E51170A75
:1081E0000BE012000501000E256F000E266F100E29
:1081F000276F000E286F12000501000E256F000E7C
:10820000266F000E276F010E286F12000501256BE7
:10821000266B276B286B05012E51130A05E005011B
:108220002E51170A0CE012000501000E216F000EFE
:10823000226F080E236F000E246F28EF41F0050116
:10824000000E216F000E226F800E236F000E246F30
:1082500021C500F122C501F123C502F124C503F1B6
:1082600025C504F126C505F127C506F128C507F186
:1082700043EC39F000C125F501C126F502C127F50F
:1082800003C128F5899A400EC76E200EC66E9E96D1
:10829000C69E030EC96EFF0E9EB602D0E82EFCD716
:1082A0009E96C69E27C5C9FFFF0E9EB602D0E82E39
:1082B000FCD79E96C69E26C5C9FFFF0E9EB602D06D
:1082C000E82EFCD79E96C69E25C5C9FFFF0E9EB61A
:1082D00002D0E82EFCD79E96C69EC952FF0E9EB6CF
:1082E00002D0E82EFCD7898AC950FF0A08E104C1F0
:1082F00025F505C126F506C127F507C128F5D89053
:10830000050124332333223321332151E00B216F24
:108310000501216793EF41F0226793EF41F0236756
:1083200093EF41F0246728EF41F00501200E252747
:10833000E86A2623E86A2723E86A28231200E86A05
:1083400005012E51130A06E005012E51170A0BE014
:10835000020E120005012851000A03E12751F00B1B
:1083600007E0010E120005012851000A01E0010E8C
:10837000120029C500F12AC501F12BC502F12CC557
:1083800003F125C504F126C505F127C506F128C569
:1083900007F1F2EC3AF003BF12009FEC41F0D8A4D1
:1083A00031EF42F0899A400EC76E200EC66E9E963F
:1083B000C69E060EC96EFF0E9EB602D0E82EFCD7F2
:1083C000898A899A9E96C69E020EC96EFF0E9EB637
:1083D00002D0E82EFCD79E96C69E27C5C9FFFF0E89
:1083E0009EB602D0E82EFCD79E96C69E26C5C9FF33
:1083F000FF0E9EB602D0E82EFCD79E96C69E25C5DF
:10840000C9FFFF0E9EB602D0E82EFCD79E96C69EF0
:10841000000EC96EFF0E9EB602D0E82EFCD7898AE8
:10842000899A9E96C69E050EC96EFF0E9EB602D014
:10843000E82EFCD79E96C69EC952FF0E9EB602D06D
:10844000E82EFCD7C9B01AEF42F0898A0501200E48
:108450002527E86A2623E86A2723E86A2823B9EF54
:1084600041F01200899A400EC76E200EC66E9E968D
:10847000C69E060EC96EFF0E9EB602D0E82EFCD731
:10848000898A899A9E96C69EC70EC96EFF0E9EB6B1
:1084900002D0E82EFCD7898A0501256B266B276B55
:1084A000286B1200899A400EC76E200EC66E9E96EB
:1084B000C69E050EC96EFF0E9EB602D0E82EFCD7F2
:1084C0009E96C69EC952FF0E9EB602D0E82EFCD7DD
:1084D000C9CF37F5898A1200899A400EC76E200EDF
:1084E000C66E9E96C69EB90EC96EFF0E9EB602D08F
:1084F000E82EFCD7898A1200899A400EC76E200E9A
:10850000C66E9E96C69EAB0EC96EFF0E9EB602D07C
:10851000E82EFCD7898AFF0EE82EFED712009FECCA
:1085200041F0D8A41200899A400EC76E200EC66E84
:108530009E96C69E030EC96EFF0E9EB602D0E82E12
:10854000FCD79E96C69E27C5C9FFFF0E9EB602D0D9
:10855000E82EFCD79E96C69E26C5C9FFFF0E9EB686
:1085600002D0E82EFCD79E96C69E25C5C9FFFF0EF9
:108570009EB602D0E82EFCD79E96C69EC952FF0E2C
:108580009EB602D0E82EFCD7898A0F01C950FF0A97
:10859000D8A40AEF46F00501FE0E376F0501FF0E65
:1085A000536FFF0E546FFF0E556FFF0E566F15A6DB
:1085B00037991586E0EC3DF0AFC538F5B0C539F513
:1085C000B1C53AF5B2C53BF5B3C53CF5B4C53DF50B
:1085D000B5C53EF50784BAC166F1BBC167F1BCC140
:1085E00068F1BDC169F14BC14FF14CC150F14DC1B2
:1085F00051F14EC152F157C159F158C15AF1000120
:108600001650010AD8B413EF43F000011650020AC5
:10861000D8B438EF43F000011650040AD8B45DEF27
:1086200043F00AEF46F00501476B486B496B4A6B14
:1086300005014B6B4C6B4D6B4E6B05014F6B506BDB
:10864000516B526B8BA0379BF4EC2BF000C1DAF12D
:1086500001C1DBF102C1DCF103C1DDF100C13FF575
:1086600001C140F502C141F503C142F57CEF43F081
:108670000501476B486B496B4A6B05014B6B4C6BB3
:108680004D6B4E6B05014F6B506B516B526BF4ECA5
:108690002BF000C1DAF101C1DBF102C1DCF103C151
:1086A000DDF1F1EC2CF000C147F501C148F502C144
:1086B00049F503C14AF50AEF46F0379BDAC13FF5A9
:1086C000DBC140F5DCC141F5DDC142F5F4EC2BF036
:1086D00000C14BF501C14CF502C14DF503C14EF58A
:1086E000F1EC2CF000C14FF501C150F502C151F57C
:1086F00003C152F57CEF43F00501616787EF43F05A
:10870000626787EF43F0636787EF43F064678BEF3F
:1087100043F0A0EF43F0DAC100F1DBC101F1DCC1AD
:1087200002F1DDC103F161C504F162C505F163C564
:1087300006F164C507F1F2EC3AF003BF0AEF46F028
:1087400059C143F55AC144F5B9C545F54AEC38F06D
:1087500036C649F537C64AF506014067B7EF43F01C
:108760004167B7EF43F04267B7EF43F04367BBEFB2
:1087700043F0CCEF43F007EC3CF00DEC3CF036C698
:1087800000F137C601F140C604F141C605F1F2EC33
:108790003AF003AF0AEF46F00101036B026B1AC611
:1087A00000F11BC601F101AFDAEF43F0FF0E026FDB
:1087B000FF0E036F0101076B066B1CC604F11DC69B
:1087C00005F105AFE8EF43F0FF0E066FFF0E076FF0
:1087D000F7EC3AF00101076B066B1EC604F11FC6E9
:1087E00005F105AFF8EF43F0FF0E066FFF0E076FC0
:1087F000F7EC3AF00101076B066B20C604F121C6C5
:1088000005F105AF08EF44F0FF0E066FFF0E076F8E
:10881000F7EC3AF0D890010103330233013300330F
:10882000D8900101033302330133003300C14BF50B
:1088300001C14CF50101036B026B22C600F123C696
:1088400001F101AF28EF44F0FF0E026FFF0E036F3E
:108850000101076B066B24C604F125C605F105AFBF
:1088600036EF44F0FF0E066FFF0E076FF7EC3AF09D
:108870000101076B066B26C604F127C605F105AF9B
:1088800046EF44F0FF0E066FFF0E076FF7EC3AF06D
:108890000101076B066B28C604F129C605F105AF77
:1088A00056EF44F0FF0E066FFF0E076FF7EC3AF03D
:1088B000D89001010333023301330033D890010112
:1088C000033302330133003300C14DF501C14EF5CE
:1088D0000101036B026B2AC600F12BC601F101AF47
:1088E00076EF44F0FF0E026FFF0E036F0101076B7E
:1088F000066B2CC604F12DC605F105AF84EF44F0DC
:10890000FF0E066FFF0E076FF7EC3AF00101076BE1
:10891000066B2EC604F12FC605F105AF94EF44F0A7
:10892000FF0E066FFF0E076FF7EC3AF00101076BC1
:10893000066B30C604F131C605F105AFA4EF44F073
:10894000FF0E066FFF0E076FF7EC3AF0D8900101AB
:108950000333023301330033D89001010333023370
:108960000133003300C14FF501C150F50101036B24
:10897000026B02C600F103C601F101AFC4EF44F07F
:10898000FF0E026FFF0E036F0101076B066B04C63B
:1089900004F105C605F105AFD2EF44F0FF0E066FF6
:1089A000FF0E076FF7EC3AF00101076B066B06C686
:1089B00004F107C605F105AFE2EF44F0FF0E066FC4
:1089C000FF0E076FF7EC3AF00101076B066B08C664
:1089D00004F109C605F105AFF2EF44F0FF0E066F92
:1089E000FF0E076FF7EC3AF0D89001010333023322
:1089F00001330033D89001010333023301330033D4
:108A000000C151F501C152F50101036B026B0AC6A9
:108A100000F10BC601F101AF12EF45F0FF0E026F3E
:108A2000FF0E036F0101076B066B0CC604F10DC648
:108A300005F105AF20EF45F0FF0E066FFF0E076F43
:108A4000F7EC3AF00101076B066B0EC604F10FC696
:108A500005F105AF30EF45F0FF0E066FFF0E076F13
:108A6000F7EC3AF00101076B066B10C604F111C672
:108A700005F105AF40EF45F0FF0E066FFF0E076FE3
:108A8000F7EC3AF0D890010103330233013300339D
:108A9000D8900101033302330133003300C153F591
:108AA00001C154F50101036B026B12C600F113C63C
:108AB00001F101AF60EF45F0FF0E026FFF0E036F93
:108AC0000101076B066B14C604F115C605F105AF6D
:108AD0006EEF45F0FF0E066FFF0E076FF7EC3AF0F2
:108AE0000101076B066B16C604F117C605F105AF49
:108AF0007EEF45F0FF0E066FFF0E076FF7EC3AF0C2
:108B00000101076B066B18C604F119C605F105AF24
:108B10008EEF45F0FF0E066FFF0E076FF7EC3AF091
:108B2000D89001010333023301330033D89001019F
:108B3000033302330133003300C155F501C156F54B
:108B40000501210E326F899A400EC76E200EC66E47
:108B50009E96C69E060EC96EFF0E9EB602D0E82EE9
:108B6000FCD7898A899A9E96C69E020EC96EFF0E10
:108B70009EB602D0E82EFCD79E96C69E27C5C9FF9A
:108B8000FF0E9EB602D0E82EFCD79E96C69E26C546
:108B9000C9FFFF0E9EB602D0E82EFCD79E96C69E59
:108BA00025C5C9FFFF0E9EB602D0E82EFCD725EEE4
:108BB00037F0322F02D0E8EF45F09E96C69EDECF0A
:108BC000C9FFFF0E9EB602D0E82EFCD7D9EF45F0C4
:108BD000898A899A9E96C69E050EC96EFF0E9EB61C
:108BE00002D0E82EFCD79E96C69EC952FF0E9EB6B6
:108BF00002D0E82EFCD7C9B0F3EF45F0898A050111
:108C0000200E2527E86A2623E86A2723E86A282316
:108C1000BEEC39F015900794120021C500F122C571
:108C200001F123C502F124C503F1899A400EC76EF4
:108C3000200EC66E9E96C69E0B0EC96EFF0E9EB689
:108C400002D0E82EFCD79E96C69E02C1C9FFFF0E39
:108C50009EB602D0E82EFCD79E96C69E01C1C9FFE3
:108C6000FF0E9EB602D0E82EFCD79E96C69E00C18F
:108C7000C9FFFF0E9EB602D0E82EFCD79E96C69E78
:108C8000C952FF0E9EB602D0E82EFCD725EE37F073
:108C90000501200E326F9E96C69EC952FF0E9EB6EB
:108CA00002D0E82EFCD7C9CFDEFF322F4BEF46F0C3
:108CB000898A1200899A400EC76E200EC66E9E9653
:108CC000C69E900EC96EFF0E9EB602D0E82EFCD74F
:108CD0009E96C69E000EC96EFF0E9EB602D0E82E6E
:108CE000FCD79E96C69E000EC96EFF0E9EB602D0A1
:108CF000E82EFCD79E96C69E000EC96EFF0E9EB64D
:108D000002D0E82EFCD79E96C69EC952FF0E9EB694
:108D100002D0E82EFCD7C9CF2DF59E96C69EC9522B
:108D2000FF0E9EB602D0E82EFCD7C9CF2EF5898A59
:108D30001200E0EC3DF005012F51010A5FE0050152
:108D40002F51020A16E005012F51030A19E005010F
:108D50002F51040A24E005012F51050A2BE00501DB
:108D60002F51060A39E005012F51070A3FE0FEEFB7
:108D700046F0602FFCEF46F05FC560F5FEEF46F071
:108D8000B0C500F101010F0E001701010051000AEA
:108D900035E001010051050A31E0FCEF46F0B0C5B5
:108DA00000F101010F0E001701010051000A26E039
:108DB000FCEF46F00501B051000A20E00501B0517A
:108DC000150A1CE00501B051300A18E00501B05148
:108DD000450A14E0FCEF46F00501B051000A0EE030
:108DE0000501B051300A0AE0FCEF46F00501B05130
:108DF000000A04E0FCEF46F0159012001580120006
:108E00008B90BEEC39F0B9C5E8FFD70802E3BEECA1
:108E100039F0B9C5E8FFC80802E3BEEC39F0B9C5BE
:108E2000E8FFB90802E3BEEC39F0B9C5E8FFAA08CB
:108E300002E3BEEC39F0B9C5E8FF9B0802E3BEECE3
:108E400039F06CEC42F0F29CF29E8B94C69AC29080
:108E5000ADEC3DF09482948C720ED36ED3A4FED709
:108E600089968A909390F29AF2949D909E909D920A
:108E70009E92F298F29286EC3FF0FF0EE8CF00F05F
:108E8000E82EFED7002EFCD7F290F286815081A802
:108E90004CEF47F0F29E0300700ED36EF296F29004
:0C8EA00015840380DFEC39F03EEF0CF08D
:10BF0000E844F926000C160C2B0C3F0C520C640C68
:10BF1000760C860C960CA50CB30CC10CCF0CDC0C6B
:06BF2000E80CF40C000C1B
:0200000400F00A
:0100C800FE39
:00000001FF
